 lcms

 Timestamp is 68fa9000 (Thu Oct 23 20:28:48 2025)

 Preferred load address is 10000000

 Start         Length     Name                   Class
 0001:00000000 00027a76H .text$mn                CODE
 0002:00000000 0000010cH .idata$5                DATA
 0002:0000010c 00000008H .00cfg                  DATA
 0002:00000114 00000004H .CRT$XCA                DATA
 0002:00000118 00000004H .CRT$XCZ                DATA
 0002:0000011c 00000004H .CRT$XIA                DATA
 0002:00000120 00000004H .CRT$XIZ                DATA
 0002:00000124 00000004H .CRT$XPA                DATA
 0002:00000128 00000004H .CRT$XPZ                DATA
 0002:0000012c 00000004H .CRT$XTA                DATA
 0002:00000130 00000010H .CRT$XTZ                DATA
 0002:00000134 00000000H .gfids$y                DATA
 0002:00000140 00004fc0H .rdata                  DATA
 0002:00005100 00000000H .rdata$CastGuardVftablesA DATA
 0002:00005100 00000000H .rdata$CastGuardVftablesC DATA
 0002:00005100 00000004H .rdata$sxdata           DATA
 0002:00005104 0000006cH .rdata$voltmd           DATA
 0002:00005170 000002e8H .rdata$zzzdbg           DATA
 0002:00005458 00000004H .rtc$IAA                DATA
 0002:0000545c 00000004H .rtc$IZZ                DATA
 0002:00005460 00000004H .rtc$TAA                DATA
 0002:00005464 00000004H .rtc$TZZ                DATA
 0002:00005468 00000088H .xdata$x                DATA
 0002:000054f0 00000268H .edata                  DATA
 0002:00005758 000000dcH .idata$2                DATA
 0002:00005834 00000014H .idata$3                DATA
 0002:00005848 0000010cH .idata$4                DATA
 0002:00005954 00000548H .idata$6                DATA
 0003:00000000 000028e8H .data                   DATA
 0003:000028e8 00001c30H .bss                    DATA
 0004:00000000 00000060H .rsrc$01                DATA
 0004:00000060 00000330H .rsrc$02                DATA

  Address         Publics by Value              Rva+Base       Lib:Object

 0000:00000000       ___AbsoluteZero            00000000     <absolute>
 0000:00000000       ___arm64x_extra_rfe_table  00000000     <absolute>
 0000:00000000       ___arm64x_extra_rfe_table_size 00000000     <absolute>
 0000:00000000       ___arm64x_native_entrypoint 00000000     <absolute>
 0000:00000000       ___arm64x_redirection_metadata 00000000     <absolute>
 0000:00000000       ___arm64x_redirection_metadata_count 00000000     <absolute>
 0000:00000000       ___dynamic_value_reloc_table 00000000     <absolute>
 0000:00000000       ___enclave_config          00000000     <absolute>
 0000:00000000       ___guard_check_icall_a64n_fptr 00000000     <absolute>
 0000:00000000       ___guard_eh_cont_count     00000000     <absolute>
 0000:00000000       ___guard_eh_cont_table     00000000     <absolute>
 0000:00000000       ___guard_fids_count        00000000     <absolute>
 0000:00000000       ___guard_fids_table        00000000     <absolute>
 0000:00000000       ___guard_iat_count         00000000     <absolute>
 0000:00000000       ___guard_iat_table         00000000     <absolute>
 0000:00000000       ___guard_longjmp_count     00000000     <absolute>
 0000:00000000       ___guard_longjmp_table     00000000     <absolute>
 0000:00000000       ___hybrid_auxiliary_delayload_iat 00000000     <absolute>
 0000:00000000       ___hybrid_auxiliary_delayload_iat_copy 00000000     <absolute>
 0000:00000000       ___hybrid_auxiliary_iat    00000000     <absolute>
 0000:00000000       ___hybrid_auxiliary_iat_copy 00000000     <absolute>
 0000:00000000       ___hybrid_code_map         00000000     <absolute>
 0000:00000000       ___hybrid_code_map_count   00000000     <absolute>
 0000:00000000       ___hybrid_image_info_bitfield 00000000     <absolute>
 0000:00000000       ___x64_code_ranges_to_entry_points 00000000     <absolute>
 0000:00000000       ___x64_code_ranges_to_entry_points_count 00000000     <absolute>
 0000:00000001       ___safe_se_handler_count   00000001     <absolute>
 0000:00000100       ___guard_flags             00000100     <absolute>
 0000:00000000       ___ImageBase               10000000     <linker-defined>
 0001:00000000       _JNI_OnLoad@8              10001000 f   LCMS.obj
 0001:00000020       _Java_sun_java2d_cmm_lcms_LCMS_colorConvert@20 10001020 f   LCMS.obj
 0001:00000240       _Java_sun_java2d_cmm_lcms_LCMS_createNativeTransform@36 10001240 f   LCMS.obj
 0001:00000460       _Java_sun_java2d_cmm_lcms_LCMS_getProfileDataNative@20 10001460 f   LCMS.obj
 0001:00000510       _Java_sun_java2d_cmm_lcms_LCMS_getProfileID@12 10001510 f   LCMS.obj
 0001:00000590       _Java_sun_java2d_cmm_lcms_LCMS_getProfileSizeNative@16 10001590 f   LCMS.obj
 0001:000005e0       _Java_sun_java2d_cmm_lcms_LCMS_getTagNative@20 100015e0 f   LCMS.obj
 0001:000007a0       _Java_sun_java2d_cmm_lcms_LCMS_initLCMS@20 100017a0 f   LCMS.obj
 0001:00000920       _Java_sun_java2d_cmm_lcms_LCMS_loadProfileNative@16 10001920 f   LCMS.obj
 0001:00000a20       _Java_sun_java2d_cmm_lcms_LCMS_setTagDataNative@24 10001a20 f   LCMS.obj
 0001:00000bc0       _LCMS_freeProfile          10001bc0 f   LCMS.obj
 0001:00000bf0       _LCMS_freeTransform        10001bf0 f   LCMS.obj
 0001:00000c00       ___local_stdio_printf_options 10001c00 f i LCMS.obj
 0001:00000c10       __snprintf                 10001c10 f i LCMS.obj
 0001:00000f40       _errorHandler              10001f40 f   LCMS.obj
 0001:00000fe0       _getILData                 10001fe0 f   LCMS.obj
 0001:000010a0       _releaseILData             100020a0 f   LCMS.obj
 0001:00001bd0       __cmsHandleExtraChannels   10002bd0 f   cmsalpha.obj
 0001:00001f60       ___local_stdio_scanf_options 10002f60 f i cmscgats.obj
 0001:00003c40       __cmsLinkProfiles          10004c40 f   cmscnvrt.obj
 0001:00003e90       @_guard_check_icall_nop@4  10004e90 f   MSVCRT:guard_support.obj
 0001:00003f20       __cmsCalloc                10004f20 f   cmserr.obj
 0001:00003f40       __cmsCreateMutex           10004f40 f   cmserr.obj
 0001:00003f60       __cmsDestroyMutex          10004f60 f   cmserr.obj
 0001:00003f80       __cmsDupMem                10004f80 f   cmserr.obj
 0001:00003fa0       __cmsFree                  10004fa0 f   cmserr.obj
 0001:00003fc0       __cmsLockMutex             10004fc0 f   cmserr.obj
 0001:00003fe0       __cmsMalloc                10004fe0 f   cmserr.obj
 0001:00004000       __cmsMallocZero            10005000 f   cmserr.obj
 0001:00004020       __cmsRealloc               10005020 f   cmserr.obj
 0001:00004040       __cmsTagSignature2String   10005040 f   cmserr.obj
 0001:00004060       __cmsUnlockMutex           10005060 f   cmserr.obj
 0001:00004080       _cmsSetLogErrorHandler     10005080 f   cmserr.obj
 0001:000040b0       _cmsSignalError            100050b0 f   cmserr.obj
 0001:00004140       _cmsfilelength             10005140 f   cmserr.obj
 0001:000050e0       _cmsBuildGamma             100060e0 f   cmsgamma.obj
 0001:00005100       _cmsBuildParametricToneCurve 10006100 f   cmsgamma.obj
 0001:000051d0       _cmsBuildSegmentedToneCurve 100061d0 f   cmsgamma.obj
 0001:00005310       _cmsBuildTabulatedToneCurve16 10006310 f   cmsgamma.obj
 0001:00005330       _cmsBuildTabulatedToneCurveFloat 10006330 f   cmsgamma.obj
 0001:00005440       _cmsDupToneCurve           10006440 f   cmsgamma.obj
 0001:00005470       _cmsEvalToneCurve16        10006470 f   cmsgamma.obj
 0001:000054a0       _cmsEvalToneCurveFloat     100064a0 f   cmsgamma.obj
 0001:00005580       _cmsFreeToneCurve          10006580 f   cmsgamma.obj
 0001:00005630       _cmsFreeToneCurveTriple    10006630 f   cmsgamma.obj
 0001:00005680       _cmsGetToneCurveParametricType 10006680 f   cmsgamma.obj
 0001:000056a0       _cmsIsToneCurveDescending  100066a0 f   cmsgamma.obj
 0001:000056c0       _cmsIsToneCurveLinear      100066c0 f   cmsgamma.obj
 0001:00005720       _cmsIsToneCurveMonotonic   10006720 f   cmsgamma.obj
 0001:000057a0       _cmsJoinToneCurve          100067a0 f   cmsgamma.obj
 0001:00005990       _cmsReverseToneCurve       10006990 f   cmsgamma.obj
 0001:000059b0       _cmsReverseToneCurveEx     100069b0 f   cmsgamma.obj
 0001:000061a0       __cmsBuildKToneCurve       100071a0 f   cmsgmt.obj
 0001:000062b0       __cmsCreateGamutCheckPipeline 100072b0 f   cmsgmt.obj
 0001:00006540       _cmsDetectTAC              10007540 f   cmsgmt.obj
 0001:00006640       __cmsFloat2Half            10007640 f   cmshalf.obj
 0001:00006670       __cmsHalf2Float            10007670 f   cmshalf.obj
 0001:0000afa0       __cmsComputeInterpParams   1000bfa0 f   cmsintrp.obj
 0001:0000b110       __cmsComputeInterpParamsEx 1000c110 f   cmsintrp.obj
 0001:0000b200       __cmsFreeInterpParams      1000c200 f   cmsintrp.obj
 0001:0000b220       __cmsSetInterpolationRoutine 1000c220 f   cmsintrp.obj
 0001:0000bc10       __cmsGetTagTrueType        1000cc10 f   cmsio0.obj
 0001:0000bcb0       __cmsReadHeader            1000ccb0 f   cmsio0.obj
 0001:0000bf50       __cmsSearchTag             1000cf50 f   cmsio0.obj
 0001:0000bfa0       __cmsWriteHeader           1000cfa0 f   cmsio0.obj
 0001:0000c200       _cmsCloseProfile           1000d200 f   cmsio0.obj
 0001:0000c310       _cmsCreateProfilePlaceholder 1000d310 f   cmsio0.obj
 0001:0000c390       _cmsGetColorSpace          1000d390 f   cmsio0.obj
 0001:0000c3a0       _cmsGetDeviceClass         1000d3a0 f   cmsio0.obj
 0001:0000c3b0       _cmsGetEncodedICCversion   1000d3b0 f   cmsio0.obj
 0001:0000c3c0       _cmsGetHeaderAttributes    1000d3c0 f   cmsio0.obj
 0001:0000c3e0       _cmsGetHeaderFlags         1000d3e0 f   cmsio0.obj
 0001:0000c3f0       _cmsGetHeaderManufacturer  1000d3f0 f   cmsio0.obj
 0001:0000c400       _cmsGetHeaderModel         1000d400 f   cmsio0.obj
 0001:0000c410       _cmsGetHeaderProfileID     1000d410 f   cmsio0.obj
 0001:0000c430       _cmsGetHeaderRenderingIntent 1000d430 f   cmsio0.obj
 0001:0000c440       _cmsGetPCS                 1000d440 f   cmsio0.obj
 0001:0000c450       _cmsGetProfileContextID    1000d450 f   cmsio0.obj
 0001:0000c460       _cmsGetProfileVersion      1000d460 f   cmsio0.obj
 0001:0000c4f0       _cmsGetTagCount            1000d4f0 f   cmsio0.obj
 0001:0000c500       _cmsGetTagSignature        1000d500 f   cmsio0.obj
 0001:0000c520       _cmsIsTag                  1000d520 f   cmsio0.obj
 0001:0000c560       _cmsLinkTag                1000d560 f   cmsio0.obj
 0001:0000c610       _cmsOpenIOhandlerFromFile  1000d610 f   cmsio0.obj
 0001:0000c770       _cmsOpenIOhandlerFromMem   1000d770 f   cmsio0.obj
 0001:0000c8d0       _cmsOpenIOhandlerFromNULL  1000d8d0 f   cmsio0.obj
 0001:0000c960       _cmsOpenProfileFromMem     1000d960 f   cmsio0.obj
 0001:0000c9b0       _cmsReadRawTag             1000d9b0 f   cmsio0.obj
 0001:0000cbf0       _cmsReadTag                1000dbf0 f   cmsio0.obj
 0001:0000ce40       _cmsSaveProfileToIOhandler 1000de40 f   cmsio0.obj
 0001:0000d020       _cmsSaveProfileToMem       1000e020 f   cmsio0.obj
 0001:0000d090       _cmsSetColorSpace          1000e090 f   cmsio0.obj
 0001:0000d0a0       _cmsSetDeviceClass         1000e0a0 f   cmsio0.obj
 0001:0000d0b0       _cmsSetEncodedICCversion   1000e0b0 f   cmsio0.obj
 0001:0000d0c0       _cmsSetHeaderAttributes    1000e0c0 f   cmsio0.obj
 0001:0000d0e0       _cmsSetHeaderFlags         1000e0e0 f   cmsio0.obj
 0001:0000d0f0       _cmsSetHeaderManufacturer  1000e0f0 f   cmsio0.obj
 0001:0000d100       _cmsSetHeaderModel         1000e100 f   cmsio0.obj
 0001:0000d110       _cmsSetHeaderProfileID     1000e110 f   cmsio0.obj
 0001:0000d130       _cmsSetHeaderRenderingIntent 1000e130 f   cmsio0.obj
 0001:0000d140       _cmsSetPCS                 1000e140 f   cmsio0.obj
 0001:0000d150       _cmsSetProfileVersion      1000e150 f   cmsio0.obj
 0001:0000d210       _cmsWriteRawTag            1000e210 f   cmsio0.obj
 0001:0000d2d0       _cmsWriteTag               1000e2d0 f   cmsio0.obj
 0001:0000d8d0       __cmsCompileProfileSequence 1000e8d0 f   cmsio1.obj
 0001:0000d9c0       __cmsReadCHAD              1000e9c0 f   cmsio1.obj
 0001:0000da70       __cmsReadDevicelinkLUT     1000ea70 f   cmsio1.obj
 0001:0000dd00       __cmsReadInputLUT          1000ed00 f   cmsio1.obj
 0001:0000e220       __cmsReadMediaWhitePoint   1000f220 f   cmsio1.obj
 0001:0000e2a0       __cmsReadOutputLUT         1000f2a0 f   cmsio1.obj
 0001:0000e580       _cmsIsCLUT                 1000f580 f   cmsio1.obj
 0001:0000e640       _cmsIsIntentSupported      1000f640 f   cmsio1.obj
 0001:0000e700       _cmsIsMatrixShaper         1000f700 f   cmsio1.obj
 0001:0000f2c0       __cmsPipelineSetOptimizationParameters 100102c0 f   cmslut.obj
 0001:0000f2f0       __cmsQuantizeVal           100102f0 f   cmslut.obj
 0001:0000f380       __cmsStageAllocIdentityCLut 10010380 f   cmslut.obj
 0001:0000f440       __cmsStageAllocIdentityCurves 10010440 f   cmslut.obj
 0001:0000f460       __cmsStageAllocLab2XYZ     10010460 f   cmslut.obj
 0001:0000f4c0       __cmsStageAllocLabV2ToV4   100104c0 f   cmslut.obj
 0001:0000f4f0       __cmsStageAllocLabV4ToV2   100104f0 f   cmslut.obj
 0001:0000f520       __cmsStageAllocPlaceholder 10010520 f   cmslut.obj
 0001:0000f580       __cmsStageAllocXYZ2Lab     10010580 f   cmslut.obj
 0001:0000f5e0       __cmsStageClipNegatives    100105e0 f   cmslut.obj
 0001:0000f630       __cmsStageGetPtrToCurveSet 10010630 f   cmslut.obj
 0001:0000f640       __cmsStageNormalizeFromLabFloat 10010640 f   cmslut.obj
 0001:0000f670       __cmsStageNormalizeFromXyzFloat 10010670 f   cmslut.obj
 0001:0000f6a0       __cmsStageNormalizeToLabFloat 100106a0 f   cmslut.obj
 0001:0000f6d0       __cmsStageNormalizeToXyzFloat 100106d0 f   cmslut.obj
 0001:0000f700       _cmsPipelineAlloc          10010700 f   cmslut.obj
 0001:0000f780       _cmsPipelineCat            10010780 f   cmslut.obj
 0001:0000f830       _cmsPipelineCheckAndRetreiveStages 10010830 f   cmslut.obj
 0001:0000f8b0       _cmsPipelineDup            100108b0 f   cmslut.obj
 0001:0000fa30       _cmsPipelineEval16         10010a30 f   cmslut.obj
 0001:0000fa50       _cmsPipelineEvalFloat      10010a50 f   cmslut.obj
 0001:0000fa60       _cmsPipelineEvalReverseFloat 10010a60 f   cmslut.obj
 0001:0000fe30       _cmsPipelineFree           10010e30 f   cmslut.obj
 0001:0000fe90       _cmsPipelineGetPtrToFirstStage 10010e90 f   cmslut.obj
 0001:0000fea0       _cmsPipelineGetPtrToLastStage 10010ea0 f   cmslut.obj
 0001:0000fec0       _cmsPipelineInputChannels  10010ec0 f   cmslut.obj
 0001:0000fec0       _cmsStageType              10010ec0 f   cmslut.obj
 0001:0000fed0       _cmsPipelineInsertStage    10010ed0 f   cmslut.obj
 0001:0000ff30       _cmsPipelineOutputChannels 10010f30 f   cmslut.obj
 0001:0000ff40       _cmsPipelineStageCount     10010f40 f   cmslut.obj
 0001:0000ff60       _cmsPipelineUnlinkStage    10010f60 f   cmslut.obj
 0001:00010010       _cmsSliceSpace16           10011010 f   cmslut.obj
 0001:000101a0       _cmsStageAllocCLut16bit    100111a0 f   cmslut.obj
 0001:00010370       _cmsStageAllocCLut16bitGranular 10011370 f   cmslut.obj
 0001:000104c0       _cmsStageAllocCLutFloatGranular 100114c0 f   cmslut.obj
 0001:000106b0       _cmsStageAllocIdentity     100116b0 f   cmslut.obj
 0001:00010700       _cmsStageAllocMatrix       10011700 f   cmslut.obj
 0001:00010970       _cmsStageAllocToneCurves   10011970 f   cmslut.obj
 0001:00010a60       _cmsStageData              10011a60 f   cmslut.obj
 0001:00010a70       _cmsStageDup               10011a70 f   cmslut.obj
 0001:00010b30       _cmsStageFree              10011b30 f   cmslut.obj
 0001:00010b50       _cmsStageInputChannels     10011b50 f   cmslut.obj
 0001:00010b60       _cmsStageNext              10011b60 f   cmslut.obj
 0001:00010b70       _cmsStageOutputChannels    10011b70 f   cmslut.obj
 0001:00010b80       _cmsStageSampleCLut16bit   10011b80 f   cmslut.obj
 0001:00010d50       __cmsMAT3eval              10011d50 f   cmsmtrx.obj
 0001:00010de0       __cmsMAT3identity          10011de0 f   cmsmtrx.obj
 0001:00010e10       __cmsMAT3inverse           10011e10 f   cmsmtrx.obj
 0001:00010f90       __cmsMAT3isIdentity        10011f90 f   cmsmtrx.obj
 0001:00011060       __cmsMAT3per               10012060 f   cmsmtrx.obj
 0001:000111d0       __cmsMAT3solve             100121d0 f   cmsmtrx.obj
 0001:000113d0       __cmsVEC3init              100123d0 f   cmsmtrx.obj
 0001:000117b0       __cmsStageAllocNamedColor  100127b0 f   cmsnamed.obj
 0001:00011800       _cmsAllocNamedColorList    10012800 f   cmsnamed.obj
 0001:000118e0       _cmsAllocProfileSequenceDescription 100128e0 f   cmsnamed.obj
 0001:00011970       _cmsAppendNamedColor       10012970 f   cmsnamed.obj
 0001:00011ac0       _cmsDictAddEntry           10012ac0 f   cmsnamed.obj
 0001:00011b90       _cmsDictAlloc              10012b90 f   cmsnamed.obj
 0001:00011bb0       _cmsDictDup                10012bb0 f   cmsnamed.obj
 0001:00011d90       _cmsDictFree               10012d90 f   cmsnamed.obj
 0001:00011e60       _cmsDictGetEntryList       10012e60 f   cmsnamed.obj
 0001:00011e60       _cmsDictNextEntry          10012e60 f   cmsnamed.obj
 0001:00011e60       _cmsNamedColorCount        10012e60 f   cmsnamed.obj
 0001:00011e70       _cmsDupNamedColorList      10012e70 f   cmsnamed.obj
 0001:00011ff0       _cmsDupProfileSequenceDescription 10012ff0 f   cmsnamed.obj
 0001:000121f0       _cmsFreeNamedColorList     100131f0 f   cmsnamed.obj
 0001:00012220       _cmsFreeProfileSequenceDescription 10013220 f   cmsnamed.obj
 0001:00012320       _cmsMLUalloc               10013320 f   cmsnamed.obj
 0001:00012380       _cmsMLUdup                 10013380 f   cmsnamed.obj
 0001:00012490       _cmsMLUfree                10013490 f   cmsnamed.obj
 0001:000124d0       _cmsMLUgetASCII            100134d0 f   cmsnamed.obj
 0001:000125e0       _cmsMLUgetWide             100135e0 f   cmsnamed.obj
 0001:000126e0       _cmsMLUsetASCII            100136e0 f   cmsnamed.obj
 0001:00012870       _cmsMLUsetWide             10013870 f   cmsnamed.obj
 0001:000128f0       _cmsNamedColorInfo         100138f0 f   cmsnamed.obj
 0001:00015930       __cmsOptimizePipeline      10016930 f   cmsopt.obj
 0001:00019ed0       __cmsFormatterIs8bit       1001aed0 f   cmspack.obj
 0001:00019ee0       __cmsFormatterIsFloat      1001aee0 f   cmspack.obj
 0001:00019ef0       __cmsGetFormatter          1001aef0 f   cmspack.obj
 0001:0001a000       _cmsFormatterForColorspaceOfProfile 1001b000 f   cmspack.obj
 0001:0001a040       __cmsEndPointsBySpace      1001b040 f   cmspcs.obj
 0001:0001a150       __cmsICCcolorSpace         1001b150 f   cmspcs.obj
 0001:0001a290       __cmsLCMScolorSpace        1001b290 f   cmspcs.obj
 0001:0001a4f0       __cmsReasonableGridpointsByColorspace 1001b4f0 f   cmspcs.obj
 0001:0001a770       _cmsChannelsOf             1001b770 f   cmspcs.obj
 0001:0001a930       _cmsDeltaE                 1001b930 f   cmspcs.obj
 0001:0001a9a0       _cmsFloat2LabEncoded       1001b9a0 f   cmspcs.obj
 0001:0001ab80       _cmsFloat2XYZEncoded       1001bb80 f   cmspcs.obj
 0001:0001ad50       _cmsLab2XYZ                1001bd50 f   cmspcs.obj
 0001:0001ae30       _cmsLabEncoded2Float       1001be30 f   cmspcs.obj
 0001:0001aea0       _cmsXYZ2Lab                1001bea0 f   cmspcs.obj
 0001:0001aff0       _cmsXYZ2xyY                1001bff0 f   cmspcs.obj
 0001:0001b040       _cmsXYZEncoded2Float       1001c040 f   cmspcs.obj
 0001:0001b080       _cmsxyY2XYZ                1001c080 f   cmspcs.obj
 0001:0001b0d0       __cms15Fixed16toDouble     1001c0d0 f   cmsplugin.obj
 0001:0001b130       __cms8Fixed8toDouble       1001c130 f   cmsplugin.obj
 0001:0001b170       __cmsAdjustEndianess32     1001c170 f   cmsplugin.obj
 0001:0001b1a0       __cmsAdjustEndianess64     1001c1a0 f   cmsplugin.obj
 0001:0001b1e0       __cmsContextGetClientChunk 1001c1e0 f   cmsplugin.obj
 0001:0001b230       __cmsDecodeDateTimeNumber  1001c230 f   cmsplugin.obj
 0001:0001b2f0       __cmsDoubleTo15Fixed16     1001c2f0 f   cmsplugin.obj
 0001:0001b330       __cmsDoubleTo8Fixed8       1001c330 f   cmsplugin.obj
 0001:0001b370       __cmsEncodeDateTimeNumber  1001c370 f   cmsplugin.obj
 0001:0001b420       __cmsGetContext            1001c420 f   cmsplugin.obj
 0001:0001b480       __cmsRead15Fixed16Number   1001c480 f   cmsplugin.obj
 0001:0001b530       __cmsReadAlignment         1001c530 f   cmsplugin.obj
 0001:0001b580       __cmsReadFloat32Number     1001c580 f   cmsplugin.obj
 0001:0001b640       __cmsReadTypeBase          1001c640 f   cmsplugin.obj
 0001:0001b6c0       __cmsReadUInt16Array       1001c6c0 f   cmsplugin.obj
 0001:0001b750       __cmsReadUInt16Number      1001c750 f   cmsplugin.obj
 0001:0001b7a0       __cmsReadUInt32Number      1001c7a0 f   cmsplugin.obj
 0001:0001b800       __cmsReadUInt64Number      1001c800 f   cmsplugin.obj
 0001:0001b870       __cmsReadUInt8Number       1001c870 f   cmsplugin.obj
 0001:0001b8b0       __cmsReadXYZNumber         1001c8b0 f   cmsplugin.obj
 0001:0001ba60       __cmsWrite15Fixed16Number  1001ca60 f   cmsplugin.obj
 0001:0001bae0       __cmsWriteAlignment        1001cae0 f   cmsplugin.obj
 0001:0001bb30       __cmsWriteFloat32Number    1001cb30 f   cmsplugin.obj
 0001:0001bb30       __cmsWriteUInt32Number     1001cb30 f   cmsplugin.obj
 0001:0001bb80       __cmsWriteTypeBase         1001cb80 f   cmsplugin.obj
 0001:0001bbf0       __cmsWriteUInt16Array      1001cbf0 f   cmsplugin.obj
 0001:0001bc60       __cmsWriteUInt16Number     1001cc60 f   cmsplugin.obj
 0001:0001bca0       __cmsWriteUInt64Number     1001cca0 f   cmsplugin.obj
 0001:0001bd10       __cmsWriteUInt8Number      1001cd10 f   cmsplugin.obj
 0001:0001bd30       __cmsWriteXYZNumber        1001cd30 f   cmsplugin.obj
 0001:0001c3b0       _cmsDetectBlackPoint       1001d3b0 f   cmssamp.obj
 0001:0001c5c0       _cmsDetectDestinationBlackPoint 1001d5c0 f   cmssamp.obj
 0001:00024590       __cmsGetTagDescriptor      10025590 f   cmstypes.obj
 0001:000245d0       __cmsGetTagTypeHandler     100255d0 f   cmstypes.obj
 0001:000247d0       _cmsCreateLab2ProfileTHR   100257d0 f   cmsvirt.obj
 0001:000248b0       _cmsCreateLab4ProfileTHR   100258b0 f   cmsvirt.obj
 0001:00024990       _cmsCreateRGBProfileTHR    10025990 f   cmsvirt.obj
 0001:00024c80       __cmsAdaptationMatrix      10025c80 f   cmswtpnt.obj
 0001:00024e90       __cmsBuildRGB2XYZtransferMatrix 10025e90 f   cmswtpnt.obj
 0001:000251e0       _cmsD50_XYZ                100261e0 f   cmswtpnt.obj
 0001:000251f0       _cmsD50_xyY                100261f0 f   cmswtpnt.obj
 0001:00025210       _cmsTempFromWhitePoint     10026210 f   cmswtpnt.obj
 0001:00025350       _cmsWhitePointFromTemp     10026350 f   cmswtpnt.obj
 0001:00026320       _cmsCreateExtendedTransform 10027320 f   cmsxform.obj
 0001:00026840       _cmsCreateMultiprofileTransform 10027840 f   cmsxform.obj
 0001:00026890       _cmsCreateMultiprofileTransformTHR 10027890 f   cmsxform.obj
 0001:00026990       _cmsCreateTransformTHR     10027990 f   cmsxform.obj
 0001:000269d0       _cmsDeleteTransform        100279d0 f   cmsxform.obj
 0001:00026a60       _cmsDoTransform            10027a60 f   cmsxform.obj
 0001:00026ada       _J2dTraceImpl              10027ada f   awt:awt.dll
 0001:00026ae0       _Disposer_AddRecord@20     10027ae0 f   awt:awt.dll
 0001:00026ae6       _JNU_ThrowByName@12        10027ae6 f   java:java.dll
 0001:00026aec       _JNU_ThrowIllegalArgumentException@8 10027aec f   java:java.dll
 0001:00026af2       ___raise_securityfailure   10027af2 f   MSVCRT:gs_report.obj
 0001:00026b1a       ___report_gsfailure        10027b1a f   MSVCRT:gs_report.obj
 0001:00026c14       ___report_rangecheckfailure 10027c14 f   MSVCRT:gs_report.obj
 0001:00026c20       ___report_securityfailure  10027c20 f   MSVCRT:gs_report.obj
 0001:00026cef       @__security_check_cookie@4 10027cef f   MSVCRT:secchk.obj
 0001:00026d00       __alloca_probe             10027d00 f   MSVCRT:chkstk.obj
 0001:00026d00       __chkstk                   10027d00 f   MSVCRT:chkstk.obj
 0001:00026d30       __dtol3                    10027d30 f   MSVCRT:ftol3.obj
 0001:00026de0       __ftol2_sse                10027de0 f   MSVCRT:ftol2.obj
 0001:00026df0       __ftoi2                    10027df0 f   MSVCRT:ftol2.obj
 0001:000271ac       __DllMainCRTStartup@12     100281ac f   MSVCRT:dll_dllmain.obj
 0001:000271cf       ___isa_available_init      100281cf f   MSVCRT:cpu_disp.obj
 0001:000273f0       ___security_init_cookie    100283f0 f   MSVCRT:gs_support.obj
 0001:0002743b       _DllMain@12                1002843b f   MSVCRT:dll_dllmain_stub.obj
 0001:0002745d       ?__scrt_initialize_type_info@@YAXXZ 1002845d f   MSVCRT:tncleanup.obj
 0001:00027469       ?__scrt_uninitialize_type_info@@YAXXZ 10028469 f   MSVCRT:tncleanup.obj
 0001:00027475       ___scrt_initialize_default_local_stdio_options 10028475 f   MSVCRT:default_local_stdio_options.obj
 0001:000274d6       ___scrt_acquire_startup_lock 100284d6 f   MSVCRT:utility.obj
 0001:00027508       ___scrt_dllmain_after_initialize_c 10028508 f   MSVCRT:utility.obj
 0001:00027533       ___scrt_dllmain_before_initialize_c 10028533 f   MSVCRT:utility.obj
 0001:00027541       ___scrt_dllmain_crt_thread_attach 10028541 f   MSVCRT:utility.obj
 0001:00027560       ___scrt_dllmain_crt_thread_detach 10028560 f   MSVCRT:utility.obj
 0001:0002756d       ___scrt_dllmain_exception_filter 1002856d f   MSVCRT:utility.obj
 0001:000275a1       ___scrt_dllmain_uninitialize_c 100285a1 f   MSVCRT:utility.obj
 0001:000275c4       ___scrt_dllmain_uninitialize_critical 100285c4 f   MSVCRT:utility.obj
 0001:000275d1       ___scrt_initialize_crt     100285d1 f   MSVCRT:utility.obj
 0001:0002760a       ___scrt_initialize_onexit_tables 1002860a f   MSVCRT:utility.obj
 0001:00027691       ___scrt_is_nonwritable_in_current_image 10028691 f   MSVCRT:utility.obj
 0001:00027725       ___scrt_release_startup_lock 10028725 f   MSVCRT:utility.obj
 0001:00027742       ___scrt_uninitialize_crt   10028742 f   MSVCRT:utility.obj
 0001:0002776a       ___scrt_get_dyn_tls_init_callback 1002876a f   MSVCRT:dyn_tls_init.obj
 0001:00027770       ___scrt_fastfail           10028770 f   MSVCRT:utility_desktop.obj
 0001:0002788b       __crt_debugger_hook        1002888b f   MSVCRT:utility_desktop.obj
 0001:00027893       __RTC_Initialize           10028893 f   MSVCRT:initsect.obj
 0001:000278bf       __RTC_Terminate            100288bf f   MSVCRT:initsect.obj
 0001:000278f0       __SEH_prolog4              100288f0 f   MSVCRT:sehprolg4.obj
 0001:00027935       __except_handler4          10028935 f   MSVCRT:chandler4gs.obj
 0001:00027964       __get_startup_argv_mode    10028964 f   MSVCRT:argv_mode.obj
 0001:00027968       ___scrt_is_ucrt_dll_in_use 10028968 f   MSVCRT:ucrt_detection.obj
 0001:00027974       _memset                    10028974 f   vcruntime:VCRUNTIME140.dll
 0001:0002797a       _memmove                   1002897a f   vcruntime:VCRUNTIME140.dll
 0001:00027980       _memcpy                    10028980 f   vcruntime:VCRUNTIME140.dll
 0001:00027986       ___std_type_info_destroy_list 10028986 f   vcruntime:VCRUNTIME140.dll
 0001:0002798c       __except_handler4_common   1002898c f   vcruntime:VCRUNTIME140.dll
 0001:00027992       _floor                     10028992 f   ucrt:api-ms-win-crt-math-l1-1-0.dll
 0001:00027998       __libm_sse2_exp_precise    10028998 f   ucrt:api-ms-win-crt-math-l1-1-0.dll
 0001:0002799e       __libm_sse2_pow_precise    1002899e f   ucrt:api-ms-win-crt-math-l1-1-0.dll
 0001:000279a4       __dclass                   100289a4 f   ucrt:api-ms-win-crt-math-l1-1-0.dll
 0001:000279aa       __libm_sse2_log10_precise  100289aa f   ucrt:api-ms-win-crt-math-l1-1-0.dll
 0001:000279b0       __libm_sse2_log_precise    100289b0 f   ucrt:api-ms-win-crt-math-l1-1-0.dll
 0001:000279b6       __libm_sse2_sqrt_precise   100289b6 f   ucrt:api-ms-win-crt-math-l1-1-0.dll
 0001:000279bc       _ceil                      100289bc f   ucrt:api-ms-win-crt-math-l1-1-0.dll
 0001:000279c2       __fdclass                  100289c2 f   ucrt:api-ms-win-crt-math-l1-1-0.dll
 0001:000279c8       __initterm                 100289c8 f   ucrt:api-ms-win-crt-runtime-l1-1-0.dll
 0001:000279ce       __initterm_e               100289ce f   ucrt:api-ms-win-crt-runtime-l1-1-0.dll
 0001:000279d4       __seh_filter_dll           100289d4 f   ucrt:api-ms-win-crt-runtime-l1-1-0.dll
 0001:000279da       __configure_narrow_argv    100289da f   ucrt:api-ms-win-crt-runtime-l1-1-0.dll
 0001:000279e0       __initialize_narrow_environment 100289e0 f   ucrt:api-ms-win-crt-runtime-l1-1-0.dll
 0001:000279e6       __initialize_onexit_table  100289e6 f   ucrt:api-ms-win-crt-runtime-l1-1-0.dll
 0001:000279ec       __execute_onexit_table     100289ec f   ucrt:api-ms-win-crt-runtime-l1-1-0.dll
 0001:000279f2       __cexit                    100289f2 f   ucrt:api-ms-win-crt-runtime-l1-1-0.dll
 0001:000279f8       ___acrt_initialize         100289f8 f   MSVCRT:ucrt_stubs.obj
 0001:000279f8       ___acrt_thread_attach      100289f8 f   MSVCRT:ucrt_stubs.obj
 0001:000279f8       ___acrt_thread_detach      100289f8 f   MSVCRT:ucrt_stubs.obj
 0001:000279f8       ___acrt_uninitialize       100289f8 f   MSVCRT:ucrt_stubs.obj
 0001:000279f8       ___acrt_uninitialize_critical 100289f8 f   MSVCRT:ucrt_stubs.obj
 0001:000279f8       ___scrt_stub_for_acrt_initialize 100289f8 f   MSVCRT:ucrt_stubs.obj
 0001:000279f8       ___scrt_stub_for_acrt_thread_attach 100289f8 f   MSVCRT:ucrt_stubs.obj
 0001:000279f8       ___scrt_stub_for_acrt_thread_detach 100289f8 f   MSVCRT:ucrt_stubs.obj
 0001:000279f8       ___scrt_stub_for_acrt_uninitialize 100289f8 f   MSVCRT:ucrt_stubs.obj
 0001:000279f8       ___scrt_stub_for_acrt_uninitialize_critical 100289f8 f   MSVCRT:ucrt_stubs.obj
 0001:000279f8       ___vcrt_initialize         100289f8 f   MSVCRT:ucrt_stubs.obj
 0001:000279f8       ___vcrt_thread_attach      100289f8 f   MSVCRT:ucrt_stubs.obj
 0001:000279f8       ___vcrt_thread_detach      100289f8 f   MSVCRT:ucrt_stubs.obj
 0001:000279f8       ___vcrt_uninitialize       100289f8 f   MSVCRT:ucrt_stubs.obj
 0001:000279f8       ___vcrt_uninitialize_critical 100289f8 f   MSVCRT:ucrt_stubs.obj
 0001:000279fb       ___scrt_stub_for_is_c_termination_complete 100289fb f   MSVCRT:ucrt_stubs.obj
 0001:000279fb       __is_c_termination_complete 100289fb f   MSVCRT:ucrt_stubs.obj
 0001:000279fe       __filter_x86_sse2_floating_point_exception 100289fe f   MSVCRT:x86_exception_filter.obj
 0001:000279fe       __filter_x86_sse2_floating_point_exception_default 100289fe f   MSVCRT:x86_exception_filter.obj
 0002:00000000       __imp__IsDebuggerPresent@0 10029000     kernel32:KERNEL32.dll
 0002:00000004       __imp__InitializeSListHead@4 10029004     kernel32:KERNEL32.dll
 0002:00000008       __imp__DisableThreadLibraryCalls@4 10029008     kernel32:KERNEL32.dll
 0002:0000000c       __imp__GetSystemTimeAsFileTime@4 1002900c     kernel32:KERNEL32.dll
 0002:00000010       __imp__InitializeCriticalSection@4 10029010     kernel32:KERNEL32.dll
 0002:00000014       __imp__EnterCriticalSection@4 10029014     kernel32:KERNEL32.dll
 0002:00000018       __imp__LeaveCriticalSection@4 10029018     kernel32:KERNEL32.dll
 0002:0000001c       __imp__DeleteCriticalSection@4 1002901c     kernel32:KERNEL32.dll
 0002:00000020       __imp__UnhandledExceptionFilter@4 10029020     kernel32:KERNEL32.dll
 0002:00000024       __imp__SetUnhandledExceptionFilter@4 10029024     kernel32:KERNEL32.dll
 0002:00000028       __imp__GetCurrentProcess@0 10029028     kernel32:KERNEL32.dll
 0002:0000002c       __imp__TerminateProcess@8  1002902c     kernel32:KERNEL32.dll
 0002:00000030       __imp__IsProcessorFeaturePresent@4 10029030     kernel32:KERNEL32.dll
 0002:00000034       __imp__QueryPerformanceCounter@4 10029034     kernel32:KERNEL32.dll
 0002:00000038       __imp__GetCurrentProcessId@0 10029038     kernel32:KERNEL32.dll
 0002:0000003c       __imp__GetCurrentThreadId@0 1002903c     kernel32:KERNEL32.dll
 0002:00000040       \177KERNEL32_NULL_THUNK_DATA 10029040     kernel32:KERNEL32.dll
 0002:00000044       __imp___except_handler4_common 10029044     vcruntime:VCRUNTIME140.dll
 0002:00000048       __imp____std_type_info_destroy_list 10029048     vcruntime:VCRUNTIME140.dll
 0002:0000004c       __imp__memcpy              1002904c     vcruntime:VCRUNTIME140.dll
 0002:00000050       __imp__memset              10029050     vcruntime:VCRUNTIME140.dll
 0002:00000054       __imp__memmove             10029054     vcruntime:VCRUNTIME140.dll
 0002:00000058       \177VCRUNTIME140_NULL_THUNK_DATA 10029058     vcruntime:VCRUNTIME140.dll
 0002:0000005c       __imp__remove              1002905c     ucrt:api-ms-win-crt-filesystem-l1-1-0.dll
 0002:00000060       \177api-ms-win-crt-filesystem-l1-1-0_NULL_THUNK_DATA 10029060     ucrt:api-ms-win-crt-filesystem-l1-1-0.dll
 0002:00000064       __imp__malloc              10029064     ucrt:api-ms-win-crt-heap-l1-1-0.dll
 0002:00000068       __imp__realloc             10029068     ucrt:api-ms-win-crt-heap-l1-1-0.dll
 0002:0000006c       __imp__free                1002906c     ucrt:api-ms-win-crt-heap-l1-1-0.dll
 0002:00000070       \177api-ms-win-crt-heap-l1-1-0_NULL_THUNK_DATA 10029070     ucrt:api-ms-win-crt-heap-l1-1-0.dll
 0002:00000074       __imp__floor               10029074     ucrt:api-ms-win-crt-math-l1-1-0.dll
 0002:00000078       __imp___libm_sse2_log_precise 10029078     ucrt:api-ms-win-crt-math-l1-1-0.dll
 0002:0000007c       __imp___libm_sse2_log10_precise 1002907c     ucrt:api-ms-win-crt-math-l1-1-0.dll
 0002:00000080       __imp___libm_sse2_exp_precise 10029080     ucrt:api-ms-win-crt-math-l1-1-0.dll
 0002:00000084       __imp___libm_sse2_pow_precise 10029084     ucrt:api-ms-win-crt-math-l1-1-0.dll
 0002:00000088       __imp___libm_sse2_sqrt_precise 10029088     ucrt:api-ms-win-crt-math-l1-1-0.dll
 0002:0000008c       __imp___fdclass            1002908c     ucrt:api-ms-win-crt-math-l1-1-0.dll
 0002:00000090       __imp__ceil                10029090     ucrt:api-ms-win-crt-math-l1-1-0.dll
 0002:00000094       __imp___dclass             10029094     ucrt:api-ms-win-crt-math-l1-1-0.dll
 0002:00000098       \177api-ms-win-crt-math-l1-1-0_NULL_THUNK_DATA 10029098     ucrt:api-ms-win-crt-math-l1-1-0.dll
 0002:0000009c       __imp___cexit              1002909c     ucrt:api-ms-win-crt-runtime-l1-1-0.dll
 0002:000000a0       __imp___execute_onexit_table 100290a0     ucrt:api-ms-win-crt-runtime-l1-1-0.dll
 0002:000000a4       __imp___initialize_onexit_table 100290a4     ucrt:api-ms-win-crt-runtime-l1-1-0.dll
 0002:000000a8       __imp___initialize_narrow_environment 100290a8     ucrt:api-ms-win-crt-runtime-l1-1-0.dll
 0002:000000ac       __imp___seh_filter_dll     100290ac     ucrt:api-ms-win-crt-runtime-l1-1-0.dll
 0002:000000b0       __imp___initterm_e         100290b0     ucrt:api-ms-win-crt-runtime-l1-1-0.dll
 0002:000000b4       __imp___configure_narrow_argv 100290b4     ucrt:api-ms-win-crt-runtime-l1-1-0.dll
 0002:000000b8       __imp___initterm           100290b8     ucrt:api-ms-win-crt-runtime-l1-1-0.dll
 0002:000000bc       \177api-ms-win-crt-runtime-l1-1-0_NULL_THUNK_DATA 100290bc     ucrt:api-ms-win-crt-runtime-l1-1-0.dll
 0002:000000c0       __imp__ftell               100290c0     ucrt:api-ms-win-crt-stdio-l1-1-0.dll
 0002:000000c4       __imp__fseek               100290c4     ucrt:api-ms-win-crt-stdio-l1-1-0.dll
 0002:000000c8       __imp__fwrite              100290c8     ucrt:api-ms-win-crt-stdio-l1-1-0.dll
 0002:000000cc       __imp__fread               100290cc     ucrt:api-ms-win-crt-stdio-l1-1-0.dll
 0002:000000d0       __imp__fopen               100290d0     ucrt:api-ms-win-crt-stdio-l1-1-0.dll
 0002:000000d4       __imp__fclose              100290d4     ucrt:api-ms-win-crt-stdio-l1-1-0.dll
 0002:000000d8       __imp____stdio_common_vsprintf 100290d8     ucrt:api-ms-win-crt-stdio-l1-1-0.dll
 0002:000000dc       \177api-ms-win-crt-stdio-l1-1-0_NULL_THUNK_DATA 100290dc     ucrt:api-ms-win-crt-stdio-l1-1-0.dll
 0002:000000e0       __imp__strncpy             100290e0     ucrt:api-ms-win-crt-string-l1-1-0.dll
 0002:000000e4       \177api-ms-win-crt-string-l1-1-0_NULL_THUNK_DATA 100290e4     ucrt:api-ms-win-crt-string-l1-1-0.dll
 0002:000000e8       __imp___time64             100290e8     ucrt:api-ms-win-crt-time-l1-1-0.dll
 0002:000000ec       __imp___gmtime64           100290ec     ucrt:api-ms-win-crt-time-l1-1-0.dll
 0002:000000f0       \177api-ms-win-crt-time-l1-1-0_NULL_THUNK_DATA 100290f0     ucrt:api-ms-win-crt-time-l1-1-0.dll
 0002:000000f4       __imp__J2dTraceImpl        100290f4     awt:awt.dll
 0002:000000f8       __imp__Disposer_AddRecord@20 100290f8     awt:awt.dll
 0002:000000fc       \177awt_NULL_THUNK_DATA    100290fc     awt:awt.dll
 0002:00000100       __imp__JNU_ThrowByName@12  10029100     java:java.dll
 0002:00000104       __imp__JNU_ThrowIllegalArgumentException@8 10029104     java:java.dll
 0002:00000108       \177java_NULL_THUNK_DATA   10029108     java:java.dll
 0002:0000010c       ___guard_check_icall_fptr  1002910c     MSVCRT:guard_support.obj
 0002:00000110       ___castguard_check_failure_os_handled_fptr 10029110     MSVCRT:guard_support.obj
 0002:00000114       ___xc_a                    10029114     MSVCRT:initializers.obj
 0002:00000118       ___xc_z                    10029118     MSVCRT:initializers.obj
 0002:0000011c       ___xi_a                    1002911c     MSVCRT:initializers.obj
 0002:00000120       ___xi_z                    10029120     MSVCRT:initializers.obj
 0002:00000124       ___xp_a                    10029124     MSVCRT:initializers.obj
 0002:00000128       ___xp_z                    10029128     MSVCRT:initializers.obj
 0002:0000012c       ___xt_a                    1002912c     MSVCRT:initializers.obj
 0002:00000130       ___xt_z                    10029130     MSVCRT:initializers.obj
 0002:00000140       ??_C@_0BC@EAADPECE@LCMS?5error?5?$CFd?3?5?$CFs@ 10029140     LCMS.obj
 0002:00000154       ??_C@_0BM@DKJNFALL@java?1awt?1color?1CMMException@ 10029154     LCMS.obj
 0002:00000170       ??_C@_0BL@NCIANLHP@getXForm?3?5iccArray?5?$DN?$DN?5NULL@ 10029170     LCMS.obj
 0002:0000018c       ??_C@_0CL@MBBNKCMD@LCMS_createNativeTransform?3?5sTr@ 1002918c     LCMS.obj
 0002:000001b8       ??_C@_0BL@NGONHNHM@Cannot?5get?5color?5transform@ 100291b8     LCMS.obj
 0002:000001d4       ??_C@_0BF@CIGEDMAF@Invalid?5profile?5data@ 100291d4     LCMS.obj
 0002:000001ec       ??_C@_0CC@DNBPCCEF@Can?5not?5access?5specified?5profil@ 100291ec     LCMS.obj
 0002:00000210       ??_C@_0BO@HCFCGEHN@Insufficient?5buffer?5capacity?4@ 10029210     LCMS.obj
 0002:00000230       ??_C@_0BN@NLFDCHLC@ICC?5Profile?5header?5not?5found@ 10029230     LCMS.obj
 0002:00000250       ??_C@_0BK@OPEDDCAA@ICC?5profile?5tag?5not?5found@ 10029250     LCMS.obj
 0002:0000026c       ??_C@_0BG@OLDFEMMB@Can?5not?5get?5tag?5data?4@ 1002926c     LCMS.obj
 0002:00000284       ??_C@_0BI@IADIMJMB@Can?5not?5write?5tag?5data?4@ 10029284     LCMS.obj
 0002:0000029c       ??_C@_0CF@MCBLFNBG@LCMS_colorConvert?3?5transform?5?$DN?$DN@ 1002929c     LCMS.obj
 0002:000002c1       ??_C@_00CNPNBAHC@@         100292c1     LCMS.obj
 0002:000002c4       ??_C@_0BJ@BAOAEIJH@Lsun?1java2d?1cmm?1Profile?$DL@ 100292c4     LCMS.obj
 0002:000002e0       ??_C@_0L@KBDEPJA@cmmProfile@ 100292e0     LCMS.obj
 0002:000002ec       ??_C@_0CA@IKDAGKDP@sun?1java2d?1cmm?1lcms?1LCMSProfile@ 100292ec     LCMS.obj
 0002:0000030c       ??_C@_01JPJNBJEM@I@        1002930c     LCMS.obj
 0002:00000310       ??_C@_0L@MNEDCAEF@renderType@ 10029310     LCMS.obj
 0002:0000031c       ??_C@_01LELAEKIP@J@        1002931c     LCMS.obj
 0002:00000320       ??_C@_02OLOABKKD@ID@       10029320     LCMS.obj
 0002:00000324       ??_C@_01POHCFINO@Z@        10029324     LCMS.obj
 0002:00000328       ??_C@_0M@BFEAFNHC@isIntPacked@ 10029328     LCMS.obj
 0002:00000334       ??_C@_08EIGIMCLE@dataType@ 10029334     LCMS.obj
 0002:00000340       ??_C@_09FECOHCAH@pixelType@ 10029340     LCMS.obj
 0002:0000034c       ??_C@_0BD@HMGGFBMH@Ljava?1lang?1Object?$DL@ 1002934c     LCMS.obj
 0002:00000360       ??_C@_09LLHCBPIG@dataArray@ 10029360     LCMS.obj
 0002:0000036c       ??_C@_05IGKADHGO@width@    1002936c     LCMS.obj
 0002:00000374       ??_C@_06LNLHEAAG@height@   10029374     LCMS.obj
 0002:0000037c       ??_C@_06KLHHMIGM@offset@   1002937c     LCMS.obj
 0002:00000384       ??_C@_0M@BFDDANOD@imageAtOnce@ 10029384     LCMS.obj
 0002:00000390       ??_C@_0O@IIJELCFP@nextRowOffset@ 10029390     LCMS.obj
 0002:000003a0       ??_C@_0CB@FCJCBIH@Unrecognized?5alpha?5channel?5widt@ 100293a0     cmsalpha.obj
 0002:000003c8       __real@3fe0000000000000    100293c8     cmsalpha.obj
 0002:000003d0       __real@406fe00000000000    100293d0     cmsalpha.obj
 0002:000003d8       __real@40dfffc000000000    100293d8     cmsalpha.obj
 0002:000003e0       __real@40efffe000000000    100293e0     cmsalpha.obj
 0002:000003e8       __real@437f0000            100293e8     cmsalpha.obj
 0002:000003ec       __real@477fff00            100293ec     cmsalpha.obj
 0002:000003f0       __real@3fb999999999999a    100293f0     cmscam02.obj
 0002:000003f8       __real@3fc999999999999a    100293f8     cmscam02.obj
 0002:00000400       __real@3fd0000000000000    10029400     cmscam02.obj
 0002:00000408       __real@3fd5555555555555    10029408     cmscam02.obj
 0002:00000410       __real@3ff0000000000000    10029410     cmscam02.obj
 0002:00000418       __real@4000000000000000    10029418     cmscam02.obj
 0002:00000420       __real@4010000000000000    10029420     cmscam02.obj
 0002:00000428       __real@4014000000000000    10029428     cmscam02.obj
 0002:00000430       __real@4059000000000000    10029430     cmscam02.obj
 0002:00000438       __real@4069000000000000    10029438     cmscam02.obj
 0002:00000440       __real@bff0000000000000    10029440     cmscam02.obj
 0002:00000450       __xmm@7fffffffffffffff7fffffffffffffff 10029450     cmscam02.obj
 0002:00000460       __xmm@80000000000000008000000000000000 10029460     cmscam02.obj
 0002:000004b0       ??_C@_08PGIMEDFK@$INCLUDE@ 100294b0     cmscgats.obj
 0002:000004bc       ??_C@_08GDKCMJME@?4INCLUDE@ 100294bc     cmscgats.obj
 0002:000004c8       ??_C@_0L@LAOBICO@BEGIN_DATA@ 100294c8     cmscgats.obj
 0002:000004d4       ??_C@_0BC@MJMHIBCL@BEGIN_DATA_FORMAT@ 100294d4     cmscgats.obj
 0002:000004e8       ??_C@_0BH@BKLCBPCO@DATA_FORMAT_IDENTIFIER@ 100294e8     cmscgats.obj
 0002:00000500       ??_C@_08PAHEKPHH@END_DATA@ 10029500     cmscgats.obj
 0002:0000050c       ??_C@_0BA@JKEAGHEK@END_DATA_FORMAT@ 1002950c     cmscgats.obj
 0002:0000051c       ??_C@_07GBPBNGKD@KEYWORD@  1002951c     cmscgats.obj
 0002:00000524       ??_C@_0BB@HDJDLEKM@NUMBER_OF_FIELDS@ 10029524     cmscgats.obj
 0002:00000538       ??_C@_0P@DOAEDAOK@NUMBER_OF_SETS@ 10029538     cmscgats.obj
 0002:00000548       ??_C@_0L@LDGMMHG@ORIGINATOR@ 10029548     cmscgats.obj
 0002:00000554       ??_C@_0BA@LGMGNJKE@FILE_DESCRIPTOR@ 10029554     cmscgats.obj
 0002:00000564       ??_C@_07BFKIKKPP@CREATED@  10029564     cmscgats.obj
 0002:0000056c       ??_C@_0L@HFJNFBAI@DESCRIPTOR@ 1002956c     cmscgats.obj
 0002:00000578       ??_C@_0BB@FHCOAJ@DIFFUSE_GEOMETRY@ 10029578     cmscgats.obj
 0002:0000058c       ??_C@_0N@LPIHKGEG@MANUFACTURER@ 1002958c     cmscgats.obj
 0002:0000059c       ??_C@_0M@NCKCGAOL@MANUFACTURE@ 1002959c     cmscgats.obj
 0002:000005a8       ??_C@_09CMIELPMF@PROD_DATE@ 100295a8     cmscgats.obj
 0002:000005b4       ??_C@_06KGGACEJG@SERIAL@   100295b4     cmscgats.obj
 0002:000005bc       ??_C@_08NCEIPHOL@MATERIAL@ 100295bc     cmscgats.obj
 0002:000005c8       ??_C@_0BA@GCECPBPC@INSTRUMENTATION@ 100295c8     cmscgats.obj
 0002:000005d8       ??_C@_0BD@EJAFHPHI@MEASUREMENT_SOURCE@ 100295d8     cmscgats.obj
 0002:000005ec       ??_C@_0BB@CCJPNIDB@PRINT_CONDITIONS@ 100295ec     cmscgats.obj
 0002:00000600       ??_C@_0P@KIIFMCBO@SAMPLE_BACKING@ 10029600     cmscgats.obj
 0002:00000610       ??_C@_09JMFPMOIF@CHISQ_DOF@ 10029610     cmscgats.obj
 0002:0000061c       ??_C@_0BF@BFDKHDLE@MEASUREMENT_GEOMETRY@ 1002961c     cmscgats.obj
 0002:00000634       ??_C@_06EKKPGGCG@FILTER@   10029634     cmscgats.obj
 0002:0000063c       ??_C@_0N@BLIEIPH@POLARIZATION@ 1002963c     cmscgats.obj
 0002:0000064c       ??_C@_0BD@PMHFGOKD@WEIGHTING_FUNCTION@ 1002964c     cmscgats.obj
 0002:00000660       ??_C@_0BI@LGGFFBDK@COMPUTATIONAL_PARAMETER@ 10029660     cmscgats.obj
 0002:00000678       ??_C@_0M@HKJIKBKL@TARGET_TYPE@ 10029678     cmscgats.obj
 0002:00000684       ??_C@_08LGFJDIAP@COLORANT@ 10029684     cmscgats.obj
 0002:00000690       ??_C@_0BB@IJIAOGIB@TABLE_DESCRIPTOR@ 10029690     cmscgats.obj
 0002:000006a4       ??_C@_0L@HJPNOMFH@TABLE_NAME@ 100296a4     cmscgats.obj
 0002:000006b0       ??_C@_09IGELLNJJ@SAMPLE_ID@ 100296b0     cmscgats.obj
 0002:000006bc       ??_C@_06IGECGLFO@STRING@   100296bc     cmscgats.obj
 0002:000006c4       ??_C@_06GBBEFBBK@CMYK_C@   100296c4     cmscgats.obj
 0002:000006cc       ??_C@_06PPJHHMJE@CMYK_M@   100296cc     cmscgats.obj
 0002:000006d4       ??_C@_06NBDJKLMB@CMYK_Y@   100296d4     cmscgats.obj
 0002:000006dc       ??_C@_06KJMNNLBC@CMYK_K@   100296dc     cmscgats.obj
 0002:000006e4       ??_C@_05ODPHEMDP@D_RED@    100296e4     cmscgats.obj
 0002:000006ec       ??_C@_07GHIFGAP@D_GREEN@   100296ec     cmscgats.obj
 0002:000006f4       ??_C@_06DLIHHAHO@D_BLUE@   100296f4     cmscgats.obj
 0002:000006fc       ??_C@_05GAAMKGJK@D_VIS@    100296fc     cmscgats.obj
 0002:00000704       ??_C@_0P@OLJLEEFM@D_MAJOR_FILTER@ 10029704     cmscgats.obj
 0002:00000714       ??_C@_05DLNILFBE@RGB_R@    10029714     cmscgats.obj
 0002:0000071c       ??_C@_05MGNFDAA@RGB_G@     1002971c     cmscgats.obj
 0002:00000724       ??_C@_05HBBKKHEF@RGB_B@    10029724     cmscgats.obj
 0002:0000072c       ??_C@_0M@LIGBHIDL@SPECTRAL_NM@ 1002972c     cmscgats.obj
 0002:00000738       ??_C@_0N@NFDMBNKK@SPECTRAL_PCT@ 10029738     cmscgats.obj
 0002:00000748       ??_C@_0N@LEJCFEG@SPECTRAL_DEC@ 10029748     cmscgats.obj
 0002:00000758       ??_C@_05CKNBCIGL@XYZ_X@    10029758     cmscgats.obj
 0002:00000760       ??_C@_05DDMKBJCK@XYZ_Y@    10029760     cmscgats.obj
 0002:00000768       ??_C@_05BIOHEKOJ@XYZ_Z@    10029768     cmscgats.obj
 0002:00000770       ??_C@_05DIGEIHIF@XYY_X@    10029770     cmscgats.obj
 0002:00000778       ??_C@_05CBHPLGME@XYY_Y@    10029778     cmscgats.obj
 0002:00000780       ??_C@_08OKLOCDPI@XYY_CAPY@ 10029780     cmscgats.obj
 0002:0000078c       ??_C@_05FJAFBMIA@LAB_L@    1002978c     cmscgats.obj
 0002:00000794       ??_C@_05OMKLGCMN@LAB_A@    10029794     cmscgats.obj
 0002:0000079c       ??_C@_05MHIGDBAO@LAB_B@    1002979c     cmscgats.obj
 0002:000007a4       ??_C@_05NOJNAAEP@LAB_C@    100297a4     cmscgats.obj
 0002:000007ac       ??_C@_05DNGJNJIE@LAB_H@    100297ac     cmscgats.obj
 0002:000007b4       ??_C@_06GOPMGMME@LAB_DE@   100297b4     cmscgats.obj
 0002:000007bc       ??_C@_09OIBLJGHC@LAB_DE_94@ 100297bc     cmscgats.obj
 0002:000007c8       ??_C@_0L@DKBFAEGH@LAB_DE_CMC@ 100297c8     cmscgats.obj
 0002:000007d4       ??_C@_0M@HPKLADL@LAB_DE_2000@ 100297d4     cmscgats.obj
 0002:000007e0       ??_C@_07HEECBDDN@MEAN_DE@  100297e0     cmscgats.obj
 0002:000007e8       ??_C@_07GJNAGIPL@STDEV_X@  100297e8     cmscgats.obj
 0002:000007f0       ??_C@_07HAMLFJLK@STDEV_Y@  100297f0     cmscgats.obj
 0002:000007f8       ??_C@_07FLOGAKHJ@STDEV_Z@  100297f8     cmscgats.obj
 0002:00000800       ??_C@_07EHHOLPKO@STDEV_L@  10029800     cmscgats.obj
 0002:00000808       ??_C@_07PCNAMBOD@STDEV_A@  10029808     cmscgats.obj
 0002:00000810       ??_C@_07NJPNJCCA@STDEV_B@  10029810     cmscgats.obj
 0002:00000818       ??_C@_08LCDEBKKI@STDEV_DE@ 10029818     cmscgats.obj
 0002:00000824       ??_C@_0M@CCEBNHDC@CHI_SQD_PAR@ 10029824     cmscgats.obj
 0002:00000830       ??_C@_0BE@FJNFGNJC@File?5?8?$CFs?8?5not?5found@ 10029830     cmscgats.obj
 0002:00000848       __real@0000000000000000    10029848     cmscgats.obj
 0002:00000850       __real@4024000000000000    10029850     cmscgats.obj
 0002:00000858       __real@4030000000000000    10029858     cmscgats.obj
 0002:00000860       ??_C@_0BE@GPNPIJJB@ColorSpace?5mismatch@ 10029860     cmscnvrt.obj
 0002:00000874       ??_C@_0BM@OKJAFLEH@Couldn?8t?5link?5?8?$CFd?8?5profiles@ 10029874     cmscnvrt.obj
 0002:00000890       ??_C@_0BI@MPGEHHCF@Unsupported?5intent?5?8?$CFd?8@ 10029890     cmscnvrt.obj
 0002:000008a8       __real@3f08001800180018    100298a8     cmscnvrt.obj
 0002:000008b0       __real@3f60624dd2f1a9fc    100298b0     cmscnvrt.obj
 0002:000008b8       __real@3f847ae147ae147b    100298b8     cmscnvrt.obj
 0002:000008c0       __xmm@3fffffe0000000003fffffe000000000 100298c0     cmscnvrt.obj
 0002:000008d0       __xmm@40efffe00000000040efffe000000000 100298d0     cmscnvrt.obj
 0002:000008e0       __xmm@7fffffff7fffffff7fffffff7fffffff 100298e0     cmscnvrt.obj
 0002:000008f0       ??_C@_0DG@DAENFMPF@Couldn?8t?5create?5tone?5curve?5of?5m@ 100298f0     cmsgamma.obj
 0002:00000928       ??_C@_0DL@NNEGPMHF@Couldn?8t?5create?5tone?5curve?5with@ 10029928     cmsgamma.obj
 0002:00000964       ??_C@_0CB@BEAJOFEK@Invalid?5parametric?5curve?5type?5?$CF@ 10029964     cmsgamma.obj
 0002:00000988       __real@3f1a36e2eb1c432d    10029988     cmsgamma.obj
 0002:00000990       __real@3f50624dd2f1a9fc    10029990     cmsgamma.obj
 0002:00000998       __real@4480f0cf00000000    10029998     cmsgamma.obj
 0002:000009a0       __real@c480f0cf00000000    100299a0     cmsgamma.obj
 0002:000009b0       __xmm@00000000000000003ff0000000000000 100299b0     cmsgamma.obj
 0002:000009c0       __xmm@41f00000000000000000000000000000 100299c0     cmsgamma.obj
 0002:000009d0       ??_C@_0DC@PJJKCCID@Wrong?5position?5of?5PCS?4?51?4?4255?5e@ 100299d0     cmsgmt.obj
 0002:00003108       ??_C@_0CO@IFGJIAPD@Too?5many?5input?5channels?5?$CI?$CFd?5cha@ 1002c108     cmsintrp.obj
 0002:00003138       ??_C@_0CM@FENLHOGF@Unsupported?5interpolation?5?$CI?$CFd?9?$DO@ 1002c138     cmsintrp.obj
 0002:00003164       __real@3089705f            1002c164     cmsintrp.obj
 0002:00003168       __real@3f800000            1002c168     cmsintrp.obj
 0002:00003170       ??_C@_0EC@HENBOIOF@Read?5from?5memory?5error?4?5Got?5?$CFd?5@ 1002c170     cmsio0.obj
 0002:000031b4       ??_C@_0CJ@PBMIOLAN@Too?5few?5data?$DL?5probably?5corrupte@ 1002c1b4     cmsio0.obj
 0002:000031e0       ??_C@_0CI@IDACEJJO@Couldn?8t?5read?5profile?5from?5NULL@ 1002c1e0     cmsio0.obj
 0002:00003208       ??_C@_0CI@FBACEILJ@Couldn?8t?5allocate?5?$CFld?5bytes?5for@ 1002c208     cmsio0.obj
 0002:00003230       ??_C@_0BJ@HOIDLEMJ@Unknown?5access?5mode?5?8?$CFc?8@ 1002c230     cmsio0.obj
 0002:0000324c       ??_C@_0DG@EGCPMNKB@Read?5error?4?5Got?5?$CFd?5bytes?0?5block@ 1002c24c     cmsio0.obj
 0002:00003284       ??_C@_0CE@FOFFALFI@Seek?5error?$DL?5probably?5corrupted?5@ 1002c284     cmsio0.obj
 0002:000032a8       ??_C@_0CE@FJNJAECP@Tell?5error?$DL?5probably?5corrupted?5@ 1002c2a8     cmsio0.obj
 0002:000032cc       ??_C@_02JDPG@rb@           1002c2cc     cmsio0.obj
 0002:000032d0       ??_C@_0BN@KEJINDNE@Cannot?5get?5size?5of?5file?5?8?$CFs?8@ 1002c2d0     cmsio0.obj
 0002:000032f0       ??_C@_02GMLFBBN@wb@        1002c2f0     cmsio0.obj
 0002:000032f4       ??_C@_0BF@IOKNJLDN@Couldn?8t?5create?5?8?$CFs?8@ 1002c2f4     cmsio0.obj
 0002:0000330c       ??_C@_0BD@JMMMDFNL@Too?5many?5tags?5?$CI?$CFd?$CJ@ 1002c30c     cmsio0.obj
 0002:00003320       ??_C@_0CG@NLDDKNPC@not?5an?5ICC?5profile?0?5invalid?5sig@ 1002c320     cmsio0.obj
 0002:00003348       ??_C@_01KDCPPGHE@r@        1002c348     cmsio0.obj
 0002:0000334c       ??_C@_0CB@FNKNDEEO@?$CIInternal?$CJ?5no?5handler?5for?5tag?5?$CF@ 1002c34c     cmsio0.obj
 0002:00003370       ??_C@_0BJ@FBKOJGB@Couldn?8t?5write?5type?5?8?$CFs?8@ 1002c370     cmsio0.obj
 0002:0000338c       ??_C@_01NOFIACDB@w@        1002c38c     cmsio0.obj
 0002:00003390       ??_C@_0BN@LCFMIKBH@Unknown?5tag?5type?5?8?$CFs?8?5found?4@ 1002c390     cmsio0.obj
 0002:000033b0       ??_C@_0BD@BIMHEJDA@Corrupted?5tag?5?8?$CFs?8@ 1002c3b0     cmsio0.obj
 0002:000033c4       ??_C@_0DH@DCJPPHOD@?8?$CFs?8?5Inconsistent?5number?5of?5ite@ 1002c3c4     cmsio0.obj
 0002:000033fc       ??_C@_0BF@BDDLIOKO@Unsupported?5tag?5?8?$CFx?8@ 1002c3fc     cmsio0.obj
 0002:00003414       ??_C@_0CD@PJOOLCAA@Unsupported?5type?5?8?$CFs?8?5for?5tag?5?8@ 1002c414     cmsio0.obj
 0002:00003438       ??_C@_0CL@BPICAPKH@Malformed?5struct?5in?5type?5?8?$CFs?8?5f@ 1002c438     cmsio0.obj
 0002:00003508       ??_C@_0BK@HHCHMIIC@Unexpected?5direction?5?$CI?$CFd?$CJ@ 1002c508     cmsio1.obj
 0002:00003530       __xmm@3fe00010001000103fe0001000100010 1002c530     cmsio1.obj
 0002:00003720       __real@00000000            1002c720     cmslut.obj
 0002:00003724       __real@3a83126f            1002c724     cmslut.obj
 0002:00003728       __real@3feff7ced9100000    1002c728     cmslut.obj
 0002:00003730       __real@3fffffe000000000    1002c730     cmslut.obj
 0002:00003738       __real@4060000000000000    1002c738     cmslut.obj
 0002:00003740       __real@4415af1d78b58c40    1002c740     cmslut.obj
 0002:00003750       __xmm@00000002000000020000000200000002 1002c750     cmslut.obj
 0002:00003760       __xmm@477fff00477fff00477fff00477fff00 1002c760     cmslut.obj
 0002:00003770       __real@3ef0001000100010    1002c770     cmsmtrx.obj
 0002:00003778       ??_C@_0BG@HHNOOACC@Color?5?$CFd?5out?5of?5range@ 1002c778     cmsnamed.obj
 0002:00003790       ??_C@_0DA@HEOCGKJM@?$CIinternal?$CJ?5Attempt?5to?5PatchLUT?5@ 1002c790     cmsopt.obj
 0002:000037c0       ??_C@_0DF@HOPCOCIH@?$CIinternal?$CJ?5?$CFd?5Channels?5are?5not?5@ 1002c7c0     cmsopt.obj
 0002:000037f8       __real@3ee4f8b580000000    1002c7f8     cmsopt.obj
 0002:00003800       __real@3f10000000000000    1002c800     cmsopt.obj
 0002:00003808       __real@3f947ae147ae147b    1002c808     cmsopt.obj
 0002:00003810       __real@40affe0000000000    1002c810     cmsopt.obj
 0002:00003818       __real@40d0000000000000    1002c818     cmsopt.obj
 0002:00003820       __real@48000000            1002c820     cmsopt.obj
 0002:00003d78       __real@40847acccccccccd    1002cd78     cmspack.obj
 0002:00003d80       __real@42c80000            1002cd80     cmspack.obj
 0002:00003d84       __real@43000000            1002cd84     cmspack.obj
 0002:00003d88       __real@4423d666            1002cd88     cmspack.obj
 0002:00003d90       __real@3f70000000000000    1002cd90     cmspcs.obj
 0002:00003d98       __real@3f747ae147ae147b    1002cd98     cmspcs.obj
 0002:00003da0       __real@3f822354d28f7cd6    1002cda0     cmspcs.obj
 0002:00003da8       __real@3fc07004ded20922    1002cda8     cmspcs.obj
 0002:00003db0       __real@3fc1a7b9611a7b96    1002cdb0     cmspcs.obj
 0002:00003db8       __real@3fca7b9611a7b961    1002cdb8     cmspcs.obj
 0002:00003dc0       __real@3ff8000000000000    1002cdc0     cmspcs.obj
 0002:00003dc8       __real@4008000000000000    1002cdc8     cmspcs.obj
 0002:00003dd0       __real@4018000000000000    1002cdd0     cmspcs.obj
 0002:00003dd8       __real@401f25ed097b425f    1002cdd8     cmspcs.obj
 0002:00003de0       __real@4049000000000000    1002cde0     cmspcs.obj
 0002:00003de8       __real@405d000000000000    1002cde8     cmspcs.obj
 0002:00003df0       __real@405fc00000000000    1002cdf0     cmspcs.obj
 0002:00003df8       __real@4070100000000000    1002cdf8     cmspcs.obj
 0002:00003e00       __real@407f400000000000    1002ce00     cmspcs.obj
 0002:00003e08       __real@40e0000000000000    1002ce08     cmspcs.obj
 0002:00003e10       __real@c060000000000000    1002ce10     cmspcs.obj
 0002:00003e18       ??_C@_0CK@PJBOBJBE@Bad?5context?5client?5?9?9?5possible?5@ 1002ce18     cmsplugin.obj
 0002:00003e48       __real@3ef0000000000000    1002ce48     cmsplugin.obj
 0002:00003e50       __real@40f0000000000000    1002ce50     cmsplugin.obj
 0002:00003e58       __real@c415af1d78b58c40    1002ce58     cmsplugin.obj
 0002:00003e60       ??_C@_02LOCGON@?$AA?$AA@   1002ce60     cmsps2.obj
 0002:00003e68       __real@3ddb7cdfd9d7bdbb    1002ce68     cmssamp.obj
 0002:00003e70       __real@3f6782d38476f2a6    1002ce70     cmssamp.obj
 0002:00003e78       __real@3f9eb851eb851eb8    1002ce78     cmssamp.obj
 0002:00003e80       __real@c049000000000000    1002ce80     cmssamp.obj
 0002:00003e90       __xmm@3f6c739e5d4db8f03f6b866e43aa79bc 1002ce90     cmssamp.obj
 0002:00003ea0       __xmm@3ff00000000000003ff0000000000000 1002cea0     cmssamp.obj
 0002:0000437c       ??_C@_11LOCGONAA@@         1002d37c     cmstypes.obj
 0002:00004380       ??_C@_0CD@KCBEPPAD@Unknown?5parametric?5curve?5type?5?8@ 1002d380     cmstypes.obj
 0002:000043a4       ??_C@_0DN@HNKCCBOO@Multisegment?5or?5Inverted?5parame@ 1002d3a4     cmstypes.obj
 0002:000043e4       ??_C@_0BN@EDFFKJHA@Unsupported?5parametric?5curve@ 1002d3e4     cmstypes.obj
 0002:00004404       ??_C@_0DJ@OPPEBCCK@multiLocalizedUnicodeType?5of?5le@ 1002d404     cmstypes.obj
 0002:00004440       ??_C@_0CL@PJACHFCE@LUT8?5needs?5256?5entries?5on?5preli@ 1002d440     cmstypes.obj
 0002:0000446c       ??_C@_0CI@FHHBLBLB@LUT?5is?5not?5suitable?5to?5be?5saved@ 1002d46c     cmstypes.obj
 0002:00004494       ??_C@_0CJ@DKPMFIFB@LUT?5is?5not?5suitable?5to?5be?5saved@ 1002d494     cmstypes.obj
 0002:000044c0       ??_C@_0BK@CIIMKOFN@Unknown?5precision?5of?5?8?$CFd?8@ 1002d4c0     cmstypes.obj
 0002:000044dc       ??_C@_0BI@HPFEABLE@Unknown?5curve?5type?5?8?$CFs?8@ 1002d4dc     cmstypes.obj
 0002:000044f4       ??_C@_0DL@BIOKLLEA@Cannot?5save?5floating?5point?5data@ 1002d4f4     cmstypes.obj
 0002:00004530       ??_C@_0CL@OHDIMNFI@LUT?5is?5not?5suitable?5to?5be?5saved@ 1002d530     cmstypes.obj
 0002:0000455c       ??_C@_0CL@ILLFOEEL@LUT?5is?5not?5suitable?5to?5be?5saved@ 1002d55c     cmstypes.obj
 0002:00004588       ??_C@_0BI@BFKMBMNC@Too?5many?5colorants?5?8?$CFd?8@ 1002d588     cmstypes.obj
 0002:000045a0       ??_C@_0BL@DNJCAEMJ@Too?5many?5named?5colors?5?8?$CFd?8@ 1002d5a0     cmstypes.obj
 0002:000045bc       ??_C@_0CB@KBIFAFKN@Too?5many?5device?5coordinates?5?8?$CFd@ 1002d5bc     cmstypes.obj
 0002:000045e0       ??_C@_02PNJEAGMK@PS@       1002d5e0     cmstypes.obj
 0002:000045e4       ??_C@_02JCKENFCN@nm@       1002d5e4     cmstypes.obj
 0002:000045e8       ??_C@_02OFPDOIKH@?$CD0@    1002d5e8     cmstypes.obj
 0002:000045ec       ??_C@_02PMOINJOG@?$CD1@    1002d5ec     cmstypes.obj
 0002:000045f0       ??_C@_02NHMFIKCF@?$CD2@    1002d5f0     cmstypes.obj
 0002:000045f4       ??_C@_02MONOLLGE@?$CD3@    1002d5f4     cmstypes.obj
 0002:000045f8       ??_C@_0CH@IABCOGPI@Unknown?5curve?5element?5type?5?8?$CFs?8@ 1002d5f8     cmstypes.obj
 0002:00004620       ??_C@_0BN@BJDFIHEG@Unknown?5MPE?5type?5?8?$CFs?8?5found?4@ 1002d620     cmstypes.obj
 0002:00004640       ??_C@_0BM@JENPCIEF@Found?5unknown?5MPE?5type?5?8?$CFs?8@ 1002d640     cmstypes.obj
 0002:0000465c       ??_C@_0CN@NNLMDML@Unsupported?5number?5of?5channels?5@ 1002d65c     cmstypes.obj
 0002:0000468c       ??_C@_0CE@HOIBEADJ@Unsupported?5bit?5depth?5for?5VCGT?5@ 1002d68c     cmstypes.obj
 0002:000046b0       ??_C@_0CD@PNHDJBNP@Unsupported?5tag?5type?5for?5VCGT?5?8@ 1002d6b0     cmstypes.obj
 0002:000046d4       ??_C@_0CJ@KPEMEFBH@Unknown?5record?5length?5in?5dictio@ 1002d6d4     cmstypes.obj
 0002:00004700       ??_C@_0BK@NPGMPAFC@Bad?5dictionary?5Name?1Value@ 1002d700     cmstypes.obj
 0002:0000471c       __real@e4078678            1002d71c     cmstypes.obj
 0002:00004720       __xmm@ffffffffffffffffffffffffffffffff 1002d720     cmstypes.obj
 0002:000048bc       ??_C@_02PLFPMECB@US@       1002d8bc     cmsvirt.obj
 0002:000048c0       ??_C@_02LFNMGJAP@en@       1002d8c0     cmsvirt.obj
 0002:000048c4       ??_C@_1DC@MIIABLA@?$AAN?$AAo?$AA?5?$AAc?$AAo?$AAp?$AAy?$AAr?$AAi?$AAg?$AAh?$AAt?$AA?0?$AA?5?$AAu@ 1002d8c4     cmsvirt.obj
 0002:000048f8       ??_C@_1BK@ODNHFBIM@?$AAR?$AAG?$AAB?$AA?5?$AAb?$AAu?$AAi?$AAl?$AAt?$AA?9?$AAi?$AAn@ 1002d8f8     cmsvirt.obj
 0002:00004914       ??_C@_1CM@HFBMKACA@?$AAL?$AAa?$AAb?$AA?5?$AAi?$AAd?$AAe?$AAn?$AAt?$AAi?$AAt?$AAy?$AA?5?$AAb?$AAu@ 1002d914     cmsvirt.obj
 0002:00004940       __real@4000cccccccccccd    1002d940     cmsvirt.obj
 0002:00004948       __real@4011333333333333    1002d948     cmsvirt.obj
 0002:00004d30       ??_C@_0CE@PHMJNENE@cmsWhitePointFromTemp?3?5invalid?5@ 1002dd30     cmswtpnt.obj
 0002:00004d58       __real@3fb95f45e0b4e11e    1002dd58     cmswtpnt.obj
 0002:00004d60       __real@3fce5753a3ec02f3    1002dd60     cmswtpnt.obj
 0002:00004d68       __real@3fcf3d74d594f26b    1002dd68     cmswtpnt.obj
 0002:00004d70       __real@3fcfad6cb5350093    1002dd70     cmswtpnt.obj
 0002:00004d78       __real@3fd199999999999a    1002dd78     cmswtpnt.obj
 0002:00004d80       __real@3ff0793dd97f62b7    1002dd80     cmswtpnt.obj
 0002:00004d88       __real@3ffe6dc5d6388659    1002dd88     cmswtpnt.obj
 0002:00004d90       __real@40000d1b71758e22    1002dd90     cmswtpnt.obj
 0002:00004d98       __real@4006f5c28f5c28f6    1002dd98     cmswtpnt.obj
 0002:00004da0       __real@4007be0ded288ce7    1002dda0     cmswtpnt.obj
 0002:00004da8       __real@40126d916872b021    1002dda8     cmswtpnt.obj
 0002:00004db0       __real@408f400000000000    1002ddb0     cmswtpnt.obj
 0002:00004db8       __real@40af400000000000    1002ddb8     cmswtpnt.obj
 0002:00004dc0       __real@40bb580000000000    1002ddc0     cmswtpnt.obj
 0002:00004dc8       __real@40d86a0000000000    1002ddc8     cmswtpnt.obj
 0002:00004dd0       __real@412e848000000000    1002ddd0     cmswtpnt.obj
 0002:00004dd8       __real@41cdcd6500000000    1002ddd8     cmswtpnt.obj
 0002:00004de0       __xmm@3fa2ca57a786c2273ffb6a7ef9db22d1 1002dde0     cmswtpnt.obj
 0002:00004df0       __xmm@3fd10cb295e9e1b13feca4a8c154c986 1002ddf0     cmswtpnt.obj
 0002:00004e00       __xmm@bfb189374bc6a7f03fa3eab367a0f909 1002de00     cmswtpnt.obj
 0002:00004e10       __xmm@bfe801a36e2eb1c4bfc4a8c154c985f0 1002de10     cmswtpnt.obj
 0002:00004e20       ??_C@_0BK@ONICMJAI@Unsupported?5raster?5format@ 1002de20     cmsxform.obj
 0002:00004e3c       ??_C@_0CB@CAFJLCLI@NULL?5input?5profiles?5on?5transfor@ 1002de3c     cmsxform.obj
 0002:00004e60       ??_C@_0CF@KNLABPMG@Wrong?5input?5color?5space?5on?5tran@ 1002de60     cmsxform.obj
 0002:00004e88       ??_C@_0CG@OGDNLNLL@Wrong?5output?5color?5space?5on?5tra@ 1002de88     cmsxform.obj
 0002:00004eb0       ??_C@_0BL@CHIHEGM@Couldn?8t?5link?5the?5profiles@ 1002deb0     cmsxform.obj
 0002:00004ecc       ??_C@_0DC@DCLBENE@Channel?5count?5doesn?8t?5match?4?5Pr@ 1002decc     cmsxform.obj
 0002:00004f00       ??_C@_0DF@JGEGJNLA@Wrong?5number?5of?5profiles?4?51?4?425@ 1002df00     cmsxform.obj
 0002:00004f38       __real@3fea6594af4f0d84    1002df38     cmsxform.obj
 0002:00004f40       __xmm@3ff00000000000003feedab9f559b3d0 1002df40     cmsxform.obj
 0002:00004f50       __xmm@40240000000000004024000000000000 1002df50     cmsxform.obj
 0002:00004f60       __xmm@bf800000bf800000bf800000bf800000 1002df60     cmsxform.obj
 0002:00004fbc       __pDefaultRawDllMain       1002dfbc     MSVCRT:dll_dllmain.obj
 0002:00004fbc       __pRawDllMain              1002dfbc     MSVCRT:dll_dllmain.obj
 0002:00004fc0       __load_config_used         1002dfc0     MSVCRT:loadcfg.obj
 0002:00005100       ___safe_se_handler_table   1002e100     <linker-defined>
 0002:00005104       ___volatile_metadata       1002e104     <linker-defined>
 0002:00005458       ___rtc_iaa                 1002e458     MSVCRT:initsect.obj
 0002:0000545c       ___rtc_izz                 1002e45c     MSVCRT:initsect.obj
 0002:00005460       ___rtc_taa                 1002e460     MSVCRT:initsect.obj
 0002:00005464       ___rtc_tzz                 1002e464     MSVCRT:initsect.obj
 0002:00005758       __IMPORT_DESCRIPTOR_awt    1002e758     awt:awt.dll
 0002:0000576c       __IMPORT_DESCRIPTOR_java   1002e76c     java:java.dll
 0002:00005780       __IMPORT_DESCRIPTOR_KERNEL32 1002e780     kernel32:KERNEL32.dll
 0002:00005794       __IMPORT_DESCRIPTOR_VCRUNTIME140 1002e794     vcruntime:VCRUNTIME140.dll
 0002:000057a8       __IMPORT_DESCRIPTOR_api-ms-win-crt-stdio-l1-1-0 1002e7a8     ucrt:api-ms-win-crt-stdio-l1-1-0.dll
 0002:000057bc       __IMPORT_DESCRIPTOR_api-ms-win-crt-heap-l1-1-0 1002e7bc     ucrt:api-ms-win-crt-heap-l1-1-0.dll
 0002:000057d0       __IMPORT_DESCRIPTOR_api-ms-win-crt-math-l1-1-0 1002e7d0     ucrt:api-ms-win-crt-math-l1-1-0.dll
 0002:000057e4       __IMPORT_DESCRIPTOR_api-ms-win-crt-string-l1-1-0 1002e7e4     ucrt:api-ms-win-crt-string-l1-1-0.dll
 0002:000057f8       __IMPORT_DESCRIPTOR_api-ms-win-crt-filesystem-l1-1-0 1002e7f8     ucrt:api-ms-win-crt-filesystem-l1-1-0.dll
 0002:0000580c       __IMPORT_DESCRIPTOR_api-ms-win-crt-time-l1-1-0 1002e80c     ucrt:api-ms-win-crt-time-l1-1-0.dll
 0002:00005820       __IMPORT_DESCRIPTOR_api-ms-win-crt-runtime-l1-1-0 1002e820     ucrt:api-ms-win-crt-runtime-l1-1-0.dll
 0002:00005834       __NULL_IMPORT_DESCRIPTOR   1002e834     awt:awt.dll
 0003:00000c80       __cmsLogErrorChunk         1002fc80     cmserr.obj
 0003:00000c84       __cmsMemPluginChunk        1002fc84     cmserr.obj
 0003:00000c9c       __cmsMutexPluginChunk      1002fc9c     cmserr.obj
 0003:00002870       __cmsAlarmCodesChunk       10031870     cmsxform.obj
 0003:00002890       __cmsAdaptationStateChunk  10031890     cmsxform.obj
 0003:000028c0       ___security_cookie_complement 100318c0     MSVCRT:gs_cookie.obj
 0003:000028c4       ___security_cookie         100318c4     MSVCRT:gs_cookie.obj
 0003:000028c8       __fltused                  100318c8     MSVCRT:fltused.obj
 0003:000028d0       ___isa_enabled             100318d0     MSVCRT:cpu_disp.obj
 0003:000028d4       ___scrt_native_dllmain_reason 100318d4     MSVCRT:utility.obj
 0003:000028e0       ___scrt_ucrt_dll_is_in_use 100318e0     MSVCRT:ucrt_stubs.obj
 0003:00002914       __cmsIntentsPluginChunk    10031914     cmscnvrt.obj
 0003:0000291c       __cmsCurvesPluginChunk     1003191c     cmsgamma.obj
 0003:00002924       __cmsInterpPluginChunk     10031924     cmsintrp.obj
 0003:0000292c       __cmsOptimizationPluginChunk 1003192c     cmsopt.obj
 0003:00002934       __cmsFormattersPluginChunk 10031934     cmspack.obj
 0003:00004170       __cmsTagTypePluginChunk    10033170     cmstypes.obj
 0003:00004174       __cmsMPETypePluginChunk    10033174     cmstypes.obj
 0003:00004178       __cmsTagPluginChunk        10033178     cmstypes.obj
 0003:000041a0       __cmsTransformPluginChunk  100331a0     cmsxform.obj
 0003:000044c8       ___isa_available           100334c8     MSVCRT:cpu_disp.obj
 0003:000044cc       ___favor                   100334cc     MSVCRT:cpu_disp.obj
 0003:000044d0       ?__type_info_root_node@@3U__type_info_node@@A 100334d0     MSVCRT:tncleanup.obj
 0003:000044d8       ___scrt_current_native_startup_state 100334d8     MSVCRT:utility.obj
 0003:000044dc       ___scrt_native_startup_lock 100334dc     MSVCRT:utility.obj
 0003:000044fc       ___scrt_debugger_hook_flag 100334fc     MSVCRT:utility_desktop.obj
 0003:00004500       ?_OptionsStorage@?1??__local_stdio_scanf_options@@9@9 10033500     <common>
 0003:00004508       ?_OptionsStorage@?1??__local_stdio_printf_options@@9@9 10033508     <common>
 0003:00004510       _javaVM                    10033510     <common>
 0003:00004514       ___dyn_tls_init_callback   10033514     <common>

 entry point at        0001:000271ac

 Static symbols

 0000:fffc9000       .debug$S                   10000000     lcms.exp
 0000:fffc9000       .debug$S                   10000000     vcruntime:VCRUNTIME140.dll
 0000:fffc9000       .debug$S                   10000000     vcruntime:VCRUNTIME140.dll
 0000:fffc9000       .debug$S                   10000000     vcruntime:VCRUNTIME140.dll
 0000:fffc9000       .debug$S                   10000000     vcruntime:VCRUNTIME140.dll
 0000:fffc9000       .debug$S                   10000000     vcruntime:VCRUNTIME140.dll
 0000:fffc9000       .debug$S                   10000000     vcruntime:VCRUNTIME140.dll
 0000:fffc9000       .debug$S                   10000000     vcruntime:VCRUNTIME140.dll
 0000:fffc9000       .debug$S                   10000000     vcruntime:VCRUNTIME140.dll
 0000:fffc9000       .debug$S                   10000000     vcruntime:VCRUNTIME140.dll
 0000:fffc9000       .debug$S                   10000000     ucrt:api-ms-win-crt-convert-l1-1-0.dll
 0002:fffd7000       .idata$6                   10000000     ucrt:api-ms-win-crt-convert-l1-1-0.dll
 0000:fffc9000       .debug$S                   10000000     ucrt:api-ms-win-crt-filesystem-l1-1-0.dll
 0000:fffc9000       .debug$S                   10000000     ucrt:api-ms-win-crt-heap-l1-1-0.dll
 0000:fffc9000       .debug$S                   10000000     ucrt:api-ms-win-crt-heap-l1-1-0.dll
 0000:fffc9000       .debug$S                   10000000     ucrt:api-ms-win-crt-heap-l1-1-0.dll
 0000:fffc9000       .debug$S                   10000000     ucrt:api-ms-win-crt-math-l1-1-0.dll
 0000:fffc9000       .debug$S                   10000000     ucrt:api-ms-win-crt-math-l1-1-0.dll
 0000:fffc9000       .debug$S                   10000000     ucrt:api-ms-win-crt-math-l1-1-0.dll
 0000:fffc9000       .debug$S                   10000000     ucrt:api-ms-win-crt-math-l1-1-0.dll
 0000:fffc9000       .debug$S                   10000000     ucrt:api-ms-win-crt-math-l1-1-0.dll
 0000:fffc9000       .debug$S                   10000000     ucrt:api-ms-win-crt-math-l1-1-0.dll
 0000:fffc9000       .debug$S                   10000000     ucrt:api-ms-win-crt-math-l1-1-0.dll
 0000:fffc9000       .debug$S                   10000000     ucrt:api-ms-win-crt-math-l1-1-0.dll
 0000:fffc9000       .debug$S                   10000000     ucrt:api-ms-win-crt-math-l1-1-0.dll
 0000:fffc9000       .debug$S                   10000000     ucrt:api-ms-win-crt-math-l1-1-0.dll
 0000:fffc9000       .debug$S                   10000000     ucrt:api-ms-win-crt-math-l1-1-0.dll
 0000:fffc9000       .debug$S                   10000000     ucrt:api-ms-win-crt-math-l1-1-0.dll
 0000:fffc9000       .debug$S                   10000000     ucrt:api-ms-win-crt-math-l1-1-0.dll
 0000:fffc9000       .debug$S                   10000000     ucrt:api-ms-win-crt-math-l1-1-0.dll
 0000:fffc9000       .debug$S                   10000000     ucrt:api-ms-win-crt-runtime-l1-1-0.dll
 0000:fffc9000       .debug$S                   10000000     ucrt:api-ms-win-crt-runtime-l1-1-0.dll
 0000:fffc9000       .debug$S                   10000000     ucrt:api-ms-win-crt-runtime-l1-1-0.dll
 0000:fffc9000       .debug$S                   10000000     ucrt:api-ms-win-crt-runtime-l1-1-0.dll
 0000:fffc9000       .debug$S                   10000000     ucrt:api-ms-win-crt-runtime-l1-1-0.dll
 0000:fffc9000       .debug$S                   10000000     ucrt:api-ms-win-crt-runtime-l1-1-0.dll
 0000:fffc9000       .debug$S                   10000000     ucrt:api-ms-win-crt-runtime-l1-1-0.dll
 0000:fffc9000       .debug$S                   10000000     ucrt:api-ms-win-crt-runtime-l1-1-0.dll
 0000:fffc9000       .debug$S                   10000000     ucrt:api-ms-win-crt-runtime-l1-1-0.dll
 0000:fffc9000       .debug$S                   10000000     ucrt:api-ms-win-crt-runtime-l1-1-0.dll
 0000:fffc9000       .debug$S                   10000000     ucrt:api-ms-win-crt-runtime-l1-1-0.dll
 0000:fffc9000       .debug$S                   10000000     ucrt:api-ms-win-crt-runtime-l1-1-0.dll
 0000:fffc9000       .debug$S                   10000000     ucrt:api-ms-win-crt-stdio-l1-1-0.dll
 0000:fffc9000       .debug$S                   10000000     ucrt:api-ms-win-crt-stdio-l1-1-0.dll
 0000:fffc9000       .debug$S                   10000000     ucrt:api-ms-win-crt-stdio-l1-1-0.dll
 0000:fffc9000       .debug$S                   10000000     ucrt:api-ms-win-crt-stdio-l1-1-0.dll
 0000:fffc9000       .debug$S                   10000000     ucrt:api-ms-win-crt-stdio-l1-1-0.dll
 0000:fffc9000       .debug$S                   10000000     ucrt:api-ms-win-crt-stdio-l1-1-0.dll
 0000:fffc9000       .debug$S                   10000000     ucrt:api-ms-win-crt-stdio-l1-1-0.dll
 0000:fffc9000       .debug$S                   10000000     ucrt:api-ms-win-crt-stdio-l1-1-0.dll
 0000:fffc9000       .debug$S                   10000000     ucrt:api-ms-win-crt-stdio-l1-1-0.dll
 0000:fffc9000       .debug$S                   10000000     ucrt:api-ms-win-crt-stdio-l1-1-0.dll
 0000:fffc9000       .debug$S                   10000000     ucrt:api-ms-win-crt-string-l1-1-0.dll
 0000:fffc9000       .debug$S                   10000000     ucrt:api-ms-win-crt-string-l1-1-0.dll
 0000:fffc9000       .debug$S                   10000000     ucrt:api-ms-win-crt-string-l1-1-0.dll
 0000:fffc9000       .debug$S                   10000000     ucrt:api-ms-win-crt-string-l1-1-0.dll
 0000:fffc9000       .debug$S                   10000000     ucrt:api-ms-win-crt-string-l1-1-0.dll
 0000:fffc9000       .debug$S                   10000000     ucrt:api-ms-win-crt-string-l1-1-0.dll
 0000:fffc9000       .debug$S                   10000000     ucrt:api-ms-win-crt-string-l1-1-0.dll
 0000:fffc9000       .debug$S                   10000000     ucrt:api-ms-win-crt-time-l1-1-0.dll
 0000:fffc9000       .debug$S                   10000000     ucrt:api-ms-win-crt-time-l1-1-0.dll
 0000:fffc9000       .debug$S                   10000000     ucrt:api-ms-win-crt-time-l1-1-0.dll
 0000:fffc9000       .debug$S                   10000000     kernel32:KERNEL32.dll
 0000:fffc9000       .debug$S                   10000000     kernel32:KERNEL32.dll
 0000:fffc9000       .debug$S                   10000000     kernel32:KERNEL32.dll
 0000:fffc9000       .debug$S                   10000000     kernel32:KERNEL32.dll
 0000:fffc9000       .debug$S                   10000000     kernel32:KERNEL32.dll
 0000:fffc9000       .debug$S                   10000000     kernel32:KERNEL32.dll
 0000:fffc9000       .debug$S                   10000000     kernel32:KERNEL32.dll
 0000:fffc9000       .debug$S                   10000000     kernel32:KERNEL32.dll
 0000:fffc9000       .debug$S                   10000000     kernel32:KERNEL32.dll
 0000:fffc9000       .debug$S                   10000000     kernel32:KERNEL32.dll
 0000:fffc9000       .debug$S                   10000000     kernel32:KERNEL32.dll
 0000:fffc9000       .debug$S                   10000000     kernel32:KERNEL32.dll
 0000:fffc9000       .debug$S                   10000000     kernel32:KERNEL32.dll
 0000:fffc9000       .debug$S                   10000000     kernel32:KERNEL32.dll
 0000:fffc9000       .debug$S                   10000000     kernel32:KERNEL32.dll
 0000:fffc9000       .debug$S                   10000000     kernel32:KERNEL32.dll
 0000:fffc9000       .debug$S                   10000000     kernel32:KERNEL32.dll
 0000:fffc9000       .debug$S                   10000000     kernel32:KERNEL32.dll
 0000:fffc9000       .debug$S                   10000000     kernel32:KERNEL32.dll
 0000:fffc9000       .debug$S                   10000000     kernel32:KERNEL32.dll
 0000:fffc9000       .debug$S                   10000000     kernel32:KERNEL32.dll
 0000:fffc9000       .debug$S                   10000000     kernel32:KERNEL32.dll
 0000:fffc9000       .debug$S                   10000000     awt:awt.dll
 0000:fffc9000       .debug$S                   10000000     awt:awt.dll
 0000:fffc9000       .debug$S                   10000000     java:java.dll
 0000:fffc9000       .debug$S                   10000000     java:java.dll
 0001:00000c50       __writeCookedTag           10001c50 f   LCMS.obj
 0001:00001084       $LN9                       10002084     LCMS.obj
 0001:00001118       $LN9                       10002118     LCMS.obj
 0001:00001130       _copy8                     10002130 f   cmsalpha.obj
 0001:00001140       _from8to16                 10002140 f   cmsalpha.obj
 0001:00001140       _from8to16SE               10002140 f   cmsalpha.obj
 0001:00001160       _from8toFLT                10002160 f   cmsalpha.obj
 0001:00001180       _from8toDBL                10002180 f   cmsalpha.obj
 0001:000011a0       _from8toHLF                100021a0 f   cmsalpha.obj
 0001:000011d0       _from16to8                 100021d0 f   cmsalpha.obj
 0001:000011f0       _from16SEto8               100021f0 f   cmsalpha.obj
 0001:00001220       _copy16                    10002220 f   cmsalpha.obj
 0001:00001230       _from16to16                10002230 f   cmsalpha.obj
 0001:00001250       _from16toFLT               10002250 f   cmsalpha.obj
 0001:00001270       _from16SEtoFLT             10002270 f   cmsalpha.obj
 0001:000012a0       _from16toDBL               100022a0 f   cmsalpha.obj
 0001:000012c0       _from16SEtoDBL             100022c0 f   cmsalpha.obj
 0001:000012f0       _from16toHLF               100022f0 f   cmsalpha.obj
 0001:00001320       _from16SEtoHLF             10002320 f   cmsalpha.obj
 0001:00001360       _fromFLTto8                10002360 f   cmsalpha.obj
 0001:000013e0       _fromFLTto16               100023e0 f   cmsalpha.obj
 0001:00001470       _fromFLTto16SE             10002470 f   cmsalpha.obj
 0001:00001510       _copy32                    10002510 f   cmsalpha.obj
 0001:00001520       _fromFLTtoDBL              10002520 f   cmsalpha.obj
 0001:00001540       _fromFLTtoHLF              10002540 f   cmsalpha.obj
 0001:00001560       _fromHLFto8                10002560 f   cmsalpha.obj
 0001:000015f0       _fromHLFto16               100025f0 f   cmsalpha.obj
 0001:00001690       _fromHLFto16SE             10002690 f   cmsalpha.obj
 0001:00001740       _fromHLFtoFLT              10002740 f   cmsalpha.obj
 0001:00001760       _fromHLFtoDBL              10002760 f   cmsalpha.obj
 0001:00001780       _fromDBLto8                10002780 f   cmsalpha.obj
 0001:00001800       _fromDBLto16               10002800 f   cmsalpha.obj
 0001:00001890       _fromDBLto16SE             10002890 f   cmsalpha.obj
 0001:00001930       _fromDBLtoFLT              10002930 f   cmsalpha.obj
 0001:00001950       _fromDBLtoHLF              10002950 f   cmsalpha.obj
 0001:00001980       _copy64                    10002980 f   cmsalpha.obj
 0001:000019a0       _ComputeComponentIncrements 100029a0 f   cmsalpha.obj
 0001:00001b70       _FormatterPos              10002b70 f   cmsalpha.obj
 0001:00001f70       _DefaultICCintents         10002f70 f   cmscnvrt.obj
 0001:000022a0       _BlackPreservingKOnlyIntents 100032a0 f   cmscnvrt.obj
 0001:0000254c       $LN54                      1000354c     cmscnvrt.obj
 0001:00002570       _BlackPreservingKPlaneIntents 10003570 f   cmscnvrt.obj
 0001:000028ec       $LN59                      100038ec     cmscnvrt.obj
 0001:00002910       _AddConversion             10003910 f   cmscnvrt.obj
 0001:00002dc0       _BlackPreservingGrayOnlySampler 10003dc0 f   cmscnvrt.obj
 0001:00002e30       _BlackPreservingSampler    10003e30 f   cmscnvrt.obj
 0001:00003300       _CHAD2Temp                 10004300 f   cmscnvrt.obj
 0001:00003440       _ComputeAbsoluteIntent     10004440 f   cmscnvrt.obj
 0001:00003880       _ComputeConversion         10004880 f   cmscnvrt.obj
 0001:00003d50       __cmsMallocDefaultFn       10004d50 f   cmserr.obj
 0001:00003d70       __cmsMallocZeroDefaultFn   10004d70 f   cmserr.obj
 0001:00003db0       __cmsFreeDefaultFn         10004db0 f   cmserr.obj
 0001:00003dd0       __cmsReallocDefaultFn      10004dd0 f   cmserr.obj
 0001:00003df0       __cmsCallocDefaultFn       10004df0 f   cmserr.obj
 0001:00003e40       __cmsDupDefaultFn          10004e40 f   cmserr.obj
 0001:00003e90       _DefaultLogErrorHandlerFunction 10004e90 f   cmserr.obj
 0001:00003ea0       _defMtxCreate              10004ea0 f   cmserr.obj
 0001:00003ed0       _defMtxDestroy             10004ed0 f   cmserr.obj
 0001:00003f00       _defMtxLock                10004f00 f   cmserr.obj
 0001:00003f10       _defMtxUnlock              10004f10 f   cmserr.obj
 0001:00004190       _DefaultEvalParametricFn   10005190 f   cmsgamma.obj
 0001:00004b1c       $LN114                     10005b1c     cmsgamma.obj
 0001:00004b70       $LN113                     10005b70     cmsgamma.obj
 0001:00004c50       _AllocateToneCurveStruct   10005c50 f   cmsgamma.obj
 0001:00004ed0       _EvalSegmentedFn           10005ed0 f   cmsgamma.obj
 0001:00005030       _GetParametricCurveByType  10006030 f   cmsgamma.obj
 0001:00005cd0       _ComputeKToLstar           10006cd0 f   cmsgmt.obj
 0001:00005f50       _EstimateTAC               10006f50 f   cmsgmt.obj
 0001:00005fe0       _GamutSampler              10006fe0 f   cmsgmt.obj
 0001:000066b0       _BilinearInterp16          100076b0 f   cmsintrp.obj
 0001:00006830       _BilinearInterpFloat       10007830 f   cmsintrp.obj
 0001:00006ab0       _Eval10Inputs              10007ab0 f   cmsintrp.obj
 0001:00006c30       _Eval10InputsFloat         10007c30 f   cmsintrp.obj
 0001:00006e40       _Eval11Inputs              10007e40 f   cmsintrp.obj
 0001:00006fc0       _Eval11InputsFloat         10007fc0 f   cmsintrp.obj
 0001:000071d0       _Eval12Inputs              100081d0 f   cmsintrp.obj
 0001:00007350       _Eval12InputsFloat         10008350 f   cmsintrp.obj
 0001:00007570       _Eval13Inputs              10008570 f   cmsintrp.obj
 0001:000076f0       _Eval13InputsFloat         100086f0 f   cmsintrp.obj
 0001:00007900       _Eval14Inputs              10008900 f   cmsintrp.obj
 0001:00007a80       _Eval14InputsFloat         10008a80 f   cmsintrp.obj
 0001:00007ca0       _Eval15Inputs              10008ca0 f   cmsintrp.obj
 0001:00007e30       _Eval15InputsFloat         10008e30 f   cmsintrp.obj
 0001:00008050       _Eval1Input                10009050 f   cmsintrp.obj
 0001:00008110       _Eval1InputFloat           10009110 f   cmsintrp.obj
 0001:00008260       _Eval4Inputs               10009260 f   cmsintrp.obj
 0001:00008960       _Eval4InputsFloat          10009960 f   cmsintrp.obj
 0001:00008b50       _Eval5Inputs               10009b50 f   cmsintrp.obj
 0001:00008cb0       _Eval5InputsFloat          10009cb0 f   cmsintrp.obj
 0001:00008eb0       _Eval6Inputs               10009eb0 f   cmsintrp.obj
 0001:00009020       _Eval6InputsFloat          1000a020 f   cmsintrp.obj
 0001:00009220       _Eval7Inputs               1000a220 f   cmsintrp.obj
 0001:00009390       _Eval7InputsFloat          1000a390 f   cmsintrp.obj
 0001:000095a0       _Eval8Inputs               1000a5a0 f   cmsintrp.obj
 0001:00009720       _Eval8InputsFloat          1000a720 f   cmsintrp.obj
 0001:00009930       _Eval9Inputs               1000a930 f   cmsintrp.obj
 0001:00009aa0       _Eval9InputsFloat          1000aaa0 f   cmsintrp.obj
 0001:00009ca0       _LinLerp1D                 1000aca0 f   cmsintrp.obj
 0001:00009d20       _LinLerp1Dfloat            1000ad20 f   cmsintrp.obj
 0001:00009e30       _TetrahedralInterp16       1000ae30 f   cmsintrp.obj
 0001:0000a330       _TetrahedralInterpFloat    1000b330 f   cmsintrp.obj
 0001:0000a840       _TrilinearInterp16         1000b840 f   cmsintrp.obj
 0001:0000ab50       _TrilinearInterpFloat      1000bb50 f   cmsintrp.obj
 0001:0000b4ec       $LN67                      1000c4ec     cmsintrp.obj
 0001:0000b530       _FileClose                 1000c530 f   cmsio0.obj
 0001:0000b560       _FileRead                  1000c560 f   cmsio0.obj
 0001:0000b5b0       _FileSeek                  1000c5b0 f   cmsio0.obj
 0001:0000b5f0       _FileTell                  1000c5f0 f   cmsio0.obj
 0001:0000b620       _FileWrite                 1000c620 f   cmsio0.obj
 0001:0000b650       _IsTypeSupported           1000c650 f   cmsio0.obj
 0001:0000b690       _MemoryClose               1000c690 f   cmsio0.obj
 0001:0000b6d0       _MemoryRead                1000c6d0 f   cmsio0.obj
 0001:0000b730       _MemorySeek                1000c730 f   cmsio0.obj
 0001:0000b760       _MemoryTell                1000c760 f   cmsio0.obj
 0001:0000b770       _MemoryWrite               1000c770 f   cmsio0.obj
 0001:0000b7d0       _NULLClose                 1000c7d0 f   cmsio0.obj
 0001:0000b800       _NULLRead                  1000c800 f   cmsio0.obj
 0001:0000b820       _NULLSeek                  1000c820 f   cmsio0.obj
 0001:0000b840       _NULLTell                  1000c840 f   cmsio0.obj
 0001:0000b850       _NULLWrite                 1000c850 f   cmsio0.obj
 0001:0000b870       _SaveTags                  1000c870 f   cmsio0.obj
 0001:0000bb90       __cmsDeleteTagByPos        1000cb90 f   cmsio0.obj
 0001:0000bc40       __cmsNewTag                1000cc40 f   cmsio0.obj
 0001:0000d550       _BuildRGBOutputMatrixShaper 1000e550 f   cmsio1.obj
 0001:0000d770       _ChangeInterpolationToTrilinear 1000e770 f   cmsio1.obj
 0001:0000d7d0       _ReadICCMatrixRGB2XYZ      1000e7d0 f   cmsio1.obj
 0001:0000e7b0       _BlessLUT                  1000f7b0 f   cmslut.obj
 0001:0000e800       _CLUTElemDup               1000f800 f   cmslut.obj
 0001:0000e8a0       _CLutElemTypeFree          1000f8a0 f   cmslut.obj
 0001:0000e8e0       _Clipper                   1000f8e0 f   cmslut.obj
 0001:0000e920       _CubeSize                  1000f920 f   cmslut.obj
 0001:0000e970       _CurveSetDup               1000f970 f   cmslut.obj
 0001:0000ea20       _CurveSetElemTypeFree      1000fa20 f   cmslut.obj
 0001:0000ea80       _EvaluateCLUTfloat         1000fa80 f   cmslut.obj
 0001:0000eaa0       _EvaluateCLUTfloatIn16     1000faa0 f   cmslut.obj
 0001:0000eb20       _EvaluateCurves            1000fb20 f   cmslut.obj
 0001:0000eb70       _EvaluateIdentity          1000fb70 f   cmslut.obj
 0001:0000eb90       _EvaluateLab2XYZ           1000fb90 f   cmslut.obj
 0001:0000ec60       _EvaluateMatrix            1000fc60 f   cmslut.obj
 0001:0000ed80       _EvaluateXYZ2Lab           1000fd80 f   cmslut.obj
 0001:0000ee50       _From16ToFloat             1000fe50 f   cmslut.obj
 0001:0000efd0       _FromFloatTo16             1000ffd0 f   cmslut.obj
 0001:0000f080       _IdentitySampler           10010080 f   cmslut.obj
 0001:0000f0b0       _MatrixElemDup             100100b0 f   cmslut.obj
 0001:0000f110       _MatrixElemTypeFree        10010110 f   cmslut.obj
 0001:0000f150       __LUTeval16                10010150 f   cmslut.obj
 0001:0000f200       __LUTevalFloat             10010200 f   cmslut.obj
 0001:00011400       _AddMLUBlock               10012400 f   cmsnamed.obj
 0001:00011540       _DupNamedColorList         10012540 f   cmsnamed.obj
 0001:00011550       _EvalNamedColor            10012550 f   cmsnamed.obj
 0001:00011650       _EvalNamedColorPCS         10012650 f   cmsnamed.obj
 0001:00011780       _FreeNamedColorList        10012780 f   cmsnamed.obj
 0001:000129c0       _OptimizeByResampling      100139c0 f   cmsopt.obj
 0001:00012ce0       _OptimizeByComputingLinearization 10013ce0 f   cmsopt.obj
 0001:000132b0       _OptimizeByJoiningCurves   100142b0 f   cmsopt.obj
 0001:000136c0       _OptimizeMatrixShaper      100146c0 f   cmsopt.obj
 0001:00013b00       _AllCurvesAreLinear        10014b00 f   cmsopt.obj
 0001:00013b50       _CurvesAlloc               10014b50 f   cmsopt.obj
 0001:00013c80       _CurvesDup                 10014c80 f   cmsopt.obj
 0001:00013cf0       _CurvesFree                10014cf0 f   cmsopt.obj
 0001:00013d30       _DupMatShaper              10014d30 f   cmsopt.obj
 0001:00013d50       _Eval16nop1D               10014d50 f   cmsopt.obj
 0001:00013d60       _FastEvaluateCurves16      10014d60 f   cmsopt.obj
 0001:00013da0       _FastEvaluateCurves8       10014da0 f   cmsopt.obj
 0001:00013de0       _FastIdentity16            10014de0 f   cmsopt.obj
 0001:00013e20       _FillFirstShaper           10014e20 f   cmsopt.obj
 0001:00013ee0       _FillSecondShaper          10014ee0 f   cmsopt.obj
 0001:00014090       _FixWhiteMisalignment      10015090 f   cmsopt.obj
 0001:00014340       _FreeMatShaper             10015340 f   cmsopt.obj
 0001:00014360       _IsDegenerated             10015360 f   cmsopt.obj
 0001:000143e0       _MatShaperEval16           100153e0 f   cmsopt.obj
 0001:00014510       _PatchLUT                  10015510 f   cmsopt.obj
 0001:000149b0       _PreOptimize               100159b0 f   cmsopt.obj
 0001:00014a90       _Prelin16dup               10015a90 f   cmsopt.obj
 0001:00014af0       _Prelin8dup                10015af0 f   cmsopt.obj
 0001:00014b10       _Prelin8free               10015b10 f   cmsopt.obj
 0001:00014b20       _PrelinEval16              10015b20 f   cmsopt.obj
 0001:00014bf0       _PrelinEval8               10015bf0 f   cmsopt.obj
 0001:00014ed0       _PrelinOpt16alloc          10015ed0 f   cmsopt.obj
 0001:00015040       _PrelinOpt16free           10016040 f   cmsopt.obj
 0001:00015070       _PrelinOpt8alloc           10016070 f   cmsopt.obj
 0001:00015210       _SlopeLimiting             10016210 f   cmsopt.obj
 0001:00015470       _XFormSampler16            10016470 f   cmsopt.obj
 0001:000156e0       __MultiplyMatrix           100166e0 f   cmsopt.obj
 0001:000158c0       __Remove2Op                100168c0 f   cmsopt.obj
 0001:00015a30       _UnrollChunkyBytes         10016a30 f   cmspack.obj
 0001:00015b40       _UnrollPlanarBytes         10016b40 f   cmspack.obj
 0001:00015c20       _Unroll4Bytes              10016c20 f   cmspack.obj
 0001:00015c70       _Unroll4BytesReverse       10016c70 f   cmspack.obj
 0001:00015cd0       _Unroll4BytesSwapFirst     10016cd0 f   cmspack.obj
 0001:00015d20       _Unroll4BytesSwap          10016d20 f   cmspack.obj
 0001:00015d70       _Unroll4BytesSwapSwapFirst 10016d70 f   cmspack.obj
 0001:00015dc0       _Unroll3Bytes              10016dc0 f   cmspack.obj
 0001:00015e00       _Unroll3BytesSkip1Swap     10016e00 f   cmspack.obj
 0001:00015e40       _Unroll3BytesSkip1SwapSwapFirst 10016e40 f   cmspack.obj
 0001:00015e80       _Unroll3BytesSkip1SwapFirst 10016e80 f   cmspack.obj
 0001:00015ec0       _Unroll3BytesSwap          10016ec0 f   cmspack.obj
 0001:00015f00       _UnrollLabV2_8             10016f00 f   cmspack.obj
 0001:00015f70       _UnrollALabV2_8            10016f70 f   cmspack.obj
 0001:00015fe0       _UnrollLabV2_16            10016fe0 f   cmspack.obj
 0001:00016030       _Unroll2Bytes              10017030 f   cmspack.obj
 0001:00016060       _Unroll1Byte               10017060 f   cmspack.obj
 0001:00016090       _Unroll1ByteSkip1          10017090 f   cmspack.obj
 0001:000160c0       _Unroll1ByteSkip2          100170c0 f   cmspack.obj
 0001:000160f0       _Unroll1ByteReversed       100170f0 f   cmspack.obj
 0001:00016120       _UnrollAnyWords            10017120 f   cmspack.obj
 0001:00016270       _UnrollPlanarWords         10017270 f   cmspack.obj
 0001:00016380       _Unroll4Words              10017380 f   cmspack.obj
 0001:000163b0       _Unroll4WordsReverse       100173b0 f   cmspack.obj
 0001:000163f0       _Unroll4WordsSwapFirst     100173f0 f   cmspack.obj
 0001:00016420       _Unroll4WordsSwap          10017420 f   cmspack.obj
 0001:00016450       _Unroll4WordsSwapSwapFirst 10017450 f   cmspack.obj
 0001:00016480       _Unroll3Words              10017480 f   cmspack.obj
 0001:000164b0       _Unroll3WordsSwap          100174b0 f   cmspack.obj
 0001:000164e0       _Unroll3WordsSkip1Swap     100174e0 f   cmspack.obj
 0001:00016510       _Unroll3WordsSkip1SwapFirst 10017510 f   cmspack.obj
 0001:00016540       _Unroll1Word               10017540 f   cmspack.obj
 0001:00016560       _Unroll1WordReversed       10017560 f   cmspack.obj
 0001:00016590       _Unroll1WordSkip3          10017590 f   cmspack.obj
 0001:000165b0       _Unroll2Words              100175b0 f   cmspack.obj
 0001:000165d0       _UnrollLabDoubleTo16       100175d0 f   cmspack.obj
 0001:00016670       _UnrollLabFloatTo16        10017670 f   cmspack.obj
 0001:00016730       _UnrollXYZDoubleTo16       10017730 f   cmspack.obj
 0001:000167d0       _UnrollXYZFloatTo16        100177d0 f   cmspack.obj
 0001:00016890       _UnrollDoubleTo16          10017890 f   cmspack.obj
 0001:00016b60       $LN63                      10017b60     cmspack.obj
 0001:00016b68       $LN62                      10017b68     cmspack.obj
 0001:00016b90       _UnrollFloatTo16           10017b90 f   cmspack.obj
 0001:00016e58       $LN63                      10017e58     cmspack.obj
 0001:00016e60       $LN62                      10017e60     cmspack.obj
 0001:00016e80       _UnrollDouble1Chan         10017e80 f   cmspack.obj
 0001:00016f10       _UnrollFloatsToFloat       10017f10 f   cmspack.obj
 0001:000170dc       $LN54                      100180dc     cmspack.obj
 0001:000170e4       $LN53                      100180e4     cmspack.obj
 0001:00017100       _UnrollDoublesToFloat      10018100 f   cmspack.obj
 0001:000172d4       $LN54                      100182d4     cmspack.obj
 0001:000172dc       $LN53                      100182dc     cmspack.obj
 0001:00017300       _UnrollLabDoubleToFloat    10018300 f   cmspack.obj
 0001:000173f0       _UnrollLabFloatToFloat     100183f0 f   cmspack.obj
 0001:000174f0       _UnrollXYZDoubleToFloat    100184f0 f   cmspack.obj
 0001:000175b0       _UnrollXYZFloatToFloat     100185b0 f   cmspack.obj
 0001:00017680       _PackAnyBytes              10018680 f   cmspack.obj
 0001:000177a0       _PackAnyWords              100187a0 f   cmspack.obj
 0001:000178e0       _PackPlanarBytes           100188e0 f   cmspack.obj
 0001:000179d0       _PackPlanarWords           100189d0 f   cmspack.obj
 0001:00017ad0       _Pack6Bytes                10018ad0 f   cmspack.obj
 0001:00017b60       _Pack6BytesSwap            10018b60 f   cmspack.obj
 0001:00017bf0       _Pack6Words                10018bf0 f   cmspack.obj
 0001:00017c30       _Pack6WordsSwap            10018c30 f   cmspack.obj
 0001:00017c70       _Pack4Bytes                10018c70 f   cmspack.obj
 0001:00017cd0       _Pack4BytesReverse         10018cd0 f   cmspack.obj
 0001:00017d40       _Pack4BytesSwapFirst       10018d40 f   cmspack.obj
 0001:00017da0       _Pack4BytesSwap            10018da0 f   cmspack.obj
 0001:00017e00       _Pack4BytesSwapSwapFirst   10018e00 f   cmspack.obj
 0001:00017e60       _Pack4Words                10018e60 f   cmspack.obj
 0001:00017e90       _Pack4WordsReverse         10018e90 f   cmspack.obj
 0001:00017ed0       _Pack4WordsSwap            10018ed0 f   cmspack.obj
 0001:00017f00       _Pack4WordsBigEndian       10018f00 f   cmspack.obj
 0001:00017f40       _PackLabV2_8               10018f40 f   cmspack.obj
 0001:00017fd0       _PackALabV2_8              10018fd0 f   cmspack.obj
 0001:00018060       _PackLabV2_16              10019060 f   cmspack.obj
 0001:000180c0       _Pack3Bytes                100190c0 f   cmspack.obj
 0001:00018110       _Pack3BytesOptimized       10019110 f   cmspack.obj
 0001:00018130       _Pack3BytesSwap            10019130 f   cmspack.obj
 0001:00018180       _Pack3BytesSwapOptimized   10019180 f   cmspack.obj
 0001:000181a0       _Pack3Words                100191a0 f   cmspack.obj
 0001:000181d0       _Pack3WordsSwap            100191d0 f   cmspack.obj
 0001:00018200       _Pack3WordsBigEndian       10019200 f   cmspack.obj
 0001:00018230       _Pack3BytesAndSkip1        10019230 f   cmspack.obj
 0001:00018280       _Pack3BytesAndSkip1Optimized 10019280 f   cmspack.obj
 0001:000182a0       _Pack3BytesAndSkip1SwapFirst 100192a0 f   cmspack.obj
 0001:000182f0       _Pack3BytesAndSkip1SwapFirstOptimized 100192f0 f   cmspack.obj
 0001:00018310       _Pack3BytesAndSkip1Swap    10019310 f   cmspack.obj
 0001:00018360       _Pack3BytesAndSkip1SwapOptimized 10019360 f   cmspack.obj
 0001:00018380       _Pack3BytesAndSkip1SwapSwapFirst 10019380 f   cmspack.obj
 0001:000183d0       _Pack3BytesAndSkip1SwapSwapFirstOptimized 100193d0 f   cmspack.obj
 0001:000183f0       _Pack3WordsAndSkip1        100193f0 f   cmspack.obj
 0001:00018420       _Pack3WordsAndSkip1Swap    10019420 f   cmspack.obj
 0001:00018450       _Pack3WordsAndSkip1SwapFirst 10019450 f   cmspack.obj
 0001:00018480       _Pack3WordsAndSkip1SwapSwapFirst 10019480 f   cmspack.obj
 0001:000184b0       _Pack1Byte                 100194b0 f   cmspack.obj
 0001:000184d0       _Pack1ByteReversed         100194d0 f   cmspack.obj
 0001:00018500       _Pack1ByteSkip1            10019500 f   cmspack.obj
 0001:00018520       _Pack1ByteSkip1SwapFirst   10019520 f   cmspack.obj
 0001:00018540       _Pack1Word                 10019540 f   cmspack.obj
 0001:00018560       _Pack1WordReversed         10019560 f   cmspack.obj
 0001:00018580       _Pack1WordBigEndian        10019580 f   cmspack.obj
 0001:000185a0       _Pack1WordSkip1            100195a0 f   cmspack.obj
 0001:000185c0       _Pack1WordSkip1SwapFirst   100195c0 f   cmspack.obj
 0001:000185e0       _PackLabDoubleFrom16       100195e0 f   cmspack.obj
 0001:00018680       _PackLabFloatFrom16        10019680 f   cmspack.obj
 0001:00018750       _PackXYZDoubleFrom16       10019750 f   cmspack.obj
 0001:00018800       _PackXYZFloatFrom16        10019800 f   cmspack.obj
 0001:000188f0       _PackDoubleFrom16          100198f0 f   cmspack.obj
 0001:00018ae4       $LN52                      10019ae4     cmspack.obj
 0001:00018aec       $LN51                      10019aec     cmspack.obj
 0001:00018b10       _PackFloatFrom16           10019b10 f   cmspack.obj
 0001:00018d04       $LN52                      10019d04     cmspack.obj
 0001:00018d0c       $LN51                      10019d0c     cmspack.obj
 0001:00018d30       _PackFloatsFromFloat       10019d30 f   cmspack.obj
 0001:00018f18       $LN53                      10019f18     cmspack.obj
 0001:00018f20       $LN52                      10019f20     cmspack.obj
 0001:00018f40       _PackDoublesFromFloat      10019f40 f   cmspack.obj
 0001:00019120       $LN52                      1001a120     cmspack.obj
 0001:00019128       $LN51                      1001a128     cmspack.obj
 0001:00019150       _PackLabFloatFromFloat     1001a150 f   cmspack.obj
 0001:00019250       _PackLabDoubleFromFloat    1001a250 f   cmspack.obj
 0001:00019340       _PackXYZFloatFromFloat     1001a340 f   cmspack.obj
 0001:00019410       _PackXYZDoubleFromFloat    1001a410 f   cmspack.obj
 0001:000194d0       _UnrollHalfTo16            1001a4d0 f   cmspack.obj
 0001:000197b8       $LN63                      1001a7b8     cmspack.obj
 0001:000197c0       $LN62                      1001a7c0     cmspack.obj
 0001:000197e0       _UnrollHalfToFloat         1001a7e0 f   cmspack.obj
 0001:000199f8       $LN54                      1001a9f8     cmspack.obj
 0001:00019a00       $LN53                      1001aa00     cmspack.obj
 0001:00019a20       _PackHalfFrom16            1001aa20 f   cmspack.obj
 0001:00019c5c       $LN53                      1001ac5c     cmspack.obj
 0001:00019c64       $LN52                      1001ac64     cmspack.obj
 0001:00019c80       _PackHalfFromFloat         1001ac80 f   cmspack.obj
 0001:00019ea4       $LN52                      1001aea4     cmspack.obj
 0001:00019eac       $LN51                      1001aeac     cmspack.obj
 0001:0001a20c       $LN36                      1001b20c     cmspcs.obj
 0001:0001a490       $LN58                      1001b490     cmspcs.obj
 0001:0001a714       $LN73                      1001b714     cmspcs.obj
 0001:0001a8dc       $LN58                      1001b8dc     cmspcs.obj
 0001:0001be90       _BlackPointAsDarkerColorant 1001ce90 f   cmssamp.obj
 0001:0001bff0       _CreateRoundtripXForm      1001cff0 f   cmssamp.obj
 0001:0001c0c0       _RootOfLeastSquaresFitQuadraticCurve 1001d0c0 f   cmssamp.obj
 0001:0001cb00       _Type_LUTB2A_Write         1001db00 f   cmstypes.obj
 0001:0001ce80       _Type_LUT16_Dup            1001de80 f   cmstypes.obj
 0001:0001ce80       _Type_LUT8_Dup             1001de80 f   cmstypes.obj
 0001:0001ce80       _Type_LUTA2B_Dup           1001de80 f   cmstypes.obj
 0001:0001ce80       _Type_LUTB2A_Dup           1001de80 f   cmstypes.obj
 0001:0001ce80       _Type_MPE_Dup              1001de80 f   cmstypes.obj
 0001:0001ce90       _Type_LUT16_Free           1001de90 f   cmstypes.obj
 0001:0001ce90       _Type_LUT8_Free            1001de90 f   cmstypes.obj
 0001:0001ce90       _Type_LUTA2B_Free          1001de90 f   cmstypes.obj
 0001:0001ce90       _Type_LUTB2A_Free          1001de90 f   cmstypes.obj
 0001:0001ce90       _Type_MPE_Free             1001de90 f   cmstypes.obj
 0001:0001cea0       _Type_ColorantTable_Read   1001dea0 f   cmstypes.obj
 0001:0001cfc0       _Type_ColorantTable_Write  1001dfc0 f   cmstypes.obj
 0001:0001d090       _Type_ColorantTable_Dup    1001e090 f   cmstypes.obj
 0001:0001d090       _Type_NamedColor_Dup       1001e090 f   cmstypes.obj
 0001:0001d0a0       _Type_ColorantTable_Free   1001e0a0 f   cmstypes.obj
 0001:0001d0a0       _Type_NamedColor_Free      1001e0a0 f   cmstypes.obj
 0001:0001d0b0       _Type_NamedColor_Read      1001e0b0 f   cmstypes.obj
 0001:0001d2b0       _Type_NamedColor_Write     1001e2b0 f   cmstypes.obj
 0001:0001d420       _Type_ProfileSequenceDesc_Read 1001e420 f   cmstypes.obj
 0001:0001d590       _Type_ProfileSequenceDesc_Write 1001e590 f   cmstypes.obj
 0001:0001d650       _Type_ProfileSequenceDesc_Dup 1001e650 f   cmstypes.obj
 0001:0001d650       _Type_ProfileSequenceId_Dup 1001e650 f   cmstypes.obj
 0001:0001d660       _Type_ProfileSequenceDesc_Free 1001e660 f   cmstypes.obj
 0001:0001d660       _Type_ProfileSequenceId_Free 1001e660 f   cmstypes.obj
 0001:0001d670       _Type_ProfileSequenceId_Read 1001e670 f   cmstypes.obj
 0001:0001d700       _Type_ProfileSequenceId_Write 1001e700 f   cmstypes.obj
 0001:0001d750       _Type_UcrBg_Read           1001e750 f   cmstypes.obj
 0001:0001d8d0       _Type_UcrBg_Write          1001e8d0 f   cmstypes.obj
 0001:0001d9b0       _Type_UcrBg_Dup            1001e9b0 f   cmstypes.obj
 0001:0001da00       _Type_UcrBg_Free           1001ea00 f   cmstypes.obj
 0001:0001da50       _Type_CrdInfo_Read         1001ea50 f   cmstypes.obj
 0001:0001db10       _Type_CrdInfo_Write        1001eb10 f   cmstypes.obj
 0001:0001db90       _Type_CrdInfo_Dup          1001eb90 f   cmstypes.obj
 0001:0001db90       _Type_MLU_Dup              1001eb90 f   cmstypes.obj
 0001:0001db90       _Type_Text_Description_Dup 1001eb90 f   cmstypes.obj
 0001:0001db90       _Type_Text_Dup             1001eb90 f   cmstypes.obj
 0001:0001dba0       _Type_CrdInfo_Free         1001eba0 f   cmstypes.obj
 0001:0001dba0       _Type_MLU_Free             1001eba0 f   cmstypes.obj
 0001:0001dba0       _Type_Text_Description_Free 1001eba0 f   cmstypes.obj
 0001:0001dba0       _Type_Text_Free            1001eba0 f   cmstypes.obj
 0001:0001dbb0       _Type_Screening_Read       1001ebb0 f   cmstypes.obj
 0001:0001dc90       _Type_Screening_Write      1001ec90 f   cmstypes.obj
 0001:0001dd30       _Type_Screening_Dup        1001ed30 f   cmstypes.obj
 0001:0001dd50       _Type_Chromaticity_Free    1001ed50 f   cmstypes.obj
 0001:0001dd50       _Type_ColorantOrderType_Free 1001ed50 f   cmstypes.obj
 0001:0001dd50       _Type_Data_Free            1001ed50 f   cmstypes.obj
 0001:0001dd50       _Type_DateTime_Free        1001ed50 f   cmstypes.obj
 0001:0001dd50       _Type_Measurement_Free     1001ed50 f   cmstypes.obj
 0001:0001dd50       _Type_S15Fixed16_Free      1001ed50 f   cmstypes.obj
 0001:0001dd50       _Type_Screening_Free       1001ed50 f   cmstypes.obj
 0001:0001dd50       _Type_Signature_Free       1001ed50 f   cmstypes.obj
 0001:0001dd50       _Type_U16Fixed16_Free      1001ed50 f   cmstypes.obj
 0001:0001dd50       _Type_ViewingConditions_Free 1001ed50 f   cmstypes.obj
 0001:0001dd50       _Type_XYZ_Free             1001ed50 f   cmstypes.obj
 0001:0001dd70       _Type_ViewingConditions_Read 1001ed70 f   cmstypes.obj
 0001:0001ddf0       _Type_ViewingConditions_Write 1001edf0 f   cmstypes.obj
 0001:0001de40       _Type_Measurement_Dup      1001ee40 f   cmstypes.obj
 0001:0001de40       _Type_ViewingConditions_Dup 1001ee40 f   cmstypes.obj
 0001:0001de60       _GenericMPEdup             1001ee60 f   cmstypes.obj
 0001:0001de70       _GenericMPEfree            1001ee70 f   cmstypes.obj
 0001:0001de80       _Type_MPEcurve_Read        1001ee80 f   cmstypes.obj
 0001:0001df90       _Type_MPEcurve_Write       1001ef90 f   cmstypes.obj
 0001:0001e000       _Type_MPEmatrix_Read       1001f000 f   cmstypes.obj
 0001:0001e180       _Type_MPEmatrix_Write      1001f180 f   cmstypes.obj
 0001:0001e240       _Type_MPEclut_Read         1001f240 f   cmstypes.obj
 0001:0001e3c0       _Type_MPEclut_Write        1001f3c0 f   cmstypes.obj
 0001:0001e4b0       _Type_MPE_Read             1001f4b0 f   cmstypes.obj
 0001:0001e5b0       _Type_MPE_Write            1001f5b0 f   cmstypes.obj
 0001:0001e8f0       _Type_vcgt_Read            1001f8f0 f   cmstypes.obj
 0001:0001ec10       _Type_vcgt_Write           1001fc10 f   cmstypes.obj
 0001:0001ee50       _Type_vcgt_Dup             1001fe50 f   cmstypes.obj
 0001:0001eea0       _Type_vcgt_Free            1001fea0 f   cmstypes.obj
 0001:0001eec0       _Type_Dictionary_Read      1001fec0 f   cmstypes.obj
 0001:0001f130       _Type_Dictionary_Write     10020130 f   cmstypes.obj
 0001:0001f3e0       _Type_Dictionary_Dup       100203e0 f   cmstypes.obj
 0001:0001f3f0       _Type_Dictionary_Free      100203f0 f   cmstypes.obj
 0001:0001f400       _Type_XYZ_Read             10020400 f   cmstypes.obj
 0001:0001f460       _Type_XYZ_Write            10020460 f   cmstypes.obj
 0001:0001f480       _Type_XYZ_Dup              10020480 f   cmstypes.obj
 0001:0001f4a0       _DecideXYZtype             100204a0 f   cmstypes.obj
 0001:0001f4b0       _Type_Chromaticity_Read    100204b0 f   cmstypes.obj
 0001:0001f610       _Type_Chromaticity_Write   10020610 f   cmstypes.obj
 0001:0001f6e0       _Type_Chromaticity_Dup     100206e0 f   cmstypes.obj
 0001:0001f700       _Type_ColorantOrderType_Read 10020700 f   cmstypes.obj
 0001:0001f790       _Type_ColorantOrderType_Write 10020790 f   cmstypes.obj
 0001:0001f800       _Type_ColorantOrderType_Dup 10020800 f   cmstypes.obj
 0001:0001f820       _Type_S15Fixed16_Read      10020820 f   cmstypes.obj
 0001:0001f8a0       _Type_S15Fixed16_Write     100208a0 f   cmstypes.obj
 0001:0001f8f0       _Type_S15Fixed16_Dup       100208f0 f   cmstypes.obj
 0001:0001f8f0       _Type_U16Fixed16_Dup       100208f0 f   cmstypes.obj
 0001:0001f910       _Type_U16Fixed16_Read      10020910 f   cmstypes.obj
 0001:0001f9b0       _Type_U16Fixed16_Write     100209b0 f   cmstypes.obj
 0001:0001fa40       _Type_Signature_Read       10020a40 f   cmstypes.obj
 0001:0001fa80       _Type_Signature_Write      10020a80 f   cmstypes.obj
 0001:0001faa0       _Type_Signature_Dup        10020aa0 f   cmstypes.obj
 0001:0001fac0       _Type_Text_Read            10020ac0 f   cmstypes.obj
 0001:0001fb80       _Type_Text_Write           10020b80 f   cmstypes.obj
 0001:0001fc00       _DecideTextType            10020c00 f   cmstypes.obj
 0001:0001fc20       _Type_Data_Read            10020c20 f   cmstypes.obj
 0001:0001fcb0       _Type_Data_Write           10020cb0 f   cmstypes.obj
 0001:0001fcf0       _Type_Data_Dup             10020cf0 f   cmstypes.obj
 0001:0001fd10       _Type_Text_Description_Read 10020d10 f   cmstypes.obj
 0001:0001fee0       _Type_Text_Description_Write 10020ee0 f   cmstypes.obj
 0001:000200e0       _DecideTextDescType        100210e0 f   cmstypes.obj
 0001:00020100       _Type_Curve_Read           10021100 f   cmstypes.obj
 0001:00020210       _Type_Curve_Write          10021210 f   cmstypes.obj
 0001:00020290       _Type_Curve_Dup            10021290 f   cmstypes.obj
 0001:00020290       _Type_ParametricCurve_Dup  10021290 f   cmstypes.obj
 0001:000202a0       _Type_Curve_Free           100212a0 f   cmstypes.obj
 0001:000202a0       _Type_ParametricCurve_Free 100212a0 f   cmstypes.obj
 0001:000202b0       _DecideCurveType           100212b0 f   cmstypes.obj
 0001:000202f0       _Type_ParametricCurve_Read 100212f0 f   cmstypes.obj
 0001:000203f0       _Type_ParametricCurve_Write 100213f0 f   cmstypes.obj
 0001:000204c0       _Type_DateTime_Read        100214c0 f   cmstypes.obj
 0001:00020550       _Type_DateTime_Write       10021550 f   cmstypes.obj
 0001:000205a0       _Type_DateTime_Dup         100215a0 f   cmstypes.obj
 0001:000205c0       _Type_Measurement_Read     100215c0 f   cmstypes.obj
 0001:00020690       _Type_Measurement_Write    10021690 f   cmstypes.obj
 0001:00020700       _Type_MLU_Read             10021700 f   cmstypes.obj
 0001:000208e0       _Type_MLU_Write            100218e0 f   cmstypes.obj
 0001:00020a20       _DecideLUTtypeA2B          10021a20 f   cmstypes.obj
 0001:00020a50       _DecideLUTtypeB2A          10021a50 f   cmstypes.obj
 0001:00020a80       _Type_LUT8_Read            10021a80 f   cmstypes.obj
 0001:00020eb0       _Type_LUT8_Write           10021eb0 f   cmstypes.obj
 0001:000211a0       _Type_LUT16_Read           100221a0 f   cmstypes.obj
 0001:000214c0       _Type_LUT16_Write          100224c0 f   cmstypes.obj
 0001:00021870       _Type_LUTA2B_Read          10022870 f   cmstypes.obj
 0001:00021a80       _Type_LUTA2B_Write         10022a80 f   cmstypes.obj
 0001:00021e10       _Type_LUTB2A_Read          10022e10 f   cmstypes.obj
 0001:00022020       _AllocArray                10023020 f   cmstypes.obj
 0001:000220f0       _AllocElem                 100230f0 f   cmstypes.obj
 0001:00022150       _FreeArray                 10023150 f   cmstypes.obj
 0001:00022240       _Read16bitTables           10023240 f   cmstypes.obj
 0001:00022350       _Read8bitTables            10023350 f   cmstypes.obj
 0001:00022550       _ReadCLUT                  10023550 f   cmstypes.obj
 0001:00022710       _ReadCountAndSting         10023710 f   cmstypes.obj
 0001:000227d0       _ReadEmbeddedText          100237d0 f   cmstypes.obj
 0001:00022960       _ReadMPECurve              10023960 f   cmstypes.obj
 0001:00022990       _ReadMPEElem               10023990 f   cmstypes.obj
 0001:00022aa0       _ReadMatrix                10023aa0 f   cmstypes.obj
 0001:00022c10       _ReadOffsetArray           10023c10 f   cmstypes.obj
 0001:00022d60       _ReadOneMLUC               10023d60 f   cmstypes.obj
 0001:00022de0       _ReadOneWChar              10023de0 f   cmstypes.obj
 0001:00022ec0       _ReadPositionTable         10023ec0 f   cmstypes.obj
 0001:00023030       _ReadSegmentedCurve        10024030 f   cmstypes.obj
 0001:00023420       _ReadSeqID                 10024420 f   cmstypes.obj
 0001:00023480       _ReadSetOfCurves           10024480 f   cmstypes.obj
 0001:00023770       _SaveDescription           10024770 f   cmstypes.obj
 0001:000237e0       _SaveOneChromaticity       100247e0 f   cmstypes.obj
 0001:00023830       _Write16bitTables          10024830 f   cmstypes.obj
 0001:00023890       _Write8bitTables           10024890 f   cmstypes.obj
 0001:00023980       _WriteCLUT                 10024980 f   cmstypes.obj
 0001:00023b20       _WriteCountAndSting        10024b20 f   cmstypes.obj
 0001:00023bb0       _WriteMPECurve             10024bb0 f   cmstypes.obj
 0001:00023bd0       _WriteMatrix               10024bd0 f   cmstypes.obj
 0001:00023cb0       _WriteOffsetArray          10024cb0 f   cmstypes.obj
 0001:00023da0       _WriteOneWChar             10024da0 f   cmstypes.obj
 0001:00023e40       _WritePositionTable        10024e40 f   cmstypes.obj
 0001:00024040       _WriteSegmentedCurve       10025040 f   cmstypes.obj
 0001:000242c0       _WriteSeqID                100252c0 f   cmstypes.obj
 0001:00024320       _WriteSetOfCurves          10025320 f   cmstypes.obj
 0001:00024610       __cmsReadWCharArray        10025610 f   cmstypes.obj
 0001:00024670       __cmsWriteWCharArray       10025670 f   cmstypes.obj
 0001:000246b0       _uipow                     100256b0 f   cmstypes.obj
 0001:00024710       _SetTextTags               10025710 f   cmsvirt.obj
 0001:00025490       _AllocEmptyTransform       10026490 f   cmsxform.obj
 0001:00025730       _CachedXFORM               10026730 f   cmsxform.obj
 0001:00025940       _CachedXFORMGamutCheck     10026940 f   cmsxform.obj
 0001:00025bb0       _FloatXFORM                10026bb0 f   cmsxform.obj
 0001:00025d40       _IsProperColorSpace        10026d40 f   cmsxform.obj
 0001:00025d90       _NullFloatXFORM            10026d90 f   cmsxform.obj
 0001:00025e90       _NullXFORM                 10026e90 f   cmsxform.obj
 0001:00025f80       _PrecalculatedXFORM        10026f80 f   cmsxform.obj
 0001:000260b0       _PrecalculatedXFORMGamutCheck 100270b0 f   cmsxform.obj
 0001:00026230       _TransformOnePixelWithGamutCheck 10027230 f   cmsxform.obj
 0001:000262b0       __cmsTransform2toTransformAdaptor 100272b0 f   cmsxform.obj
 0001:00026d00       $$000000                   10027d00     MSVCRT:chkstk.obj
 0001:00026d14       cs10                       10027d14     MSVCRT:chkstk.obj
 0001:00026d22       cs20                       10027d22     MSVCRT:chkstk.obj
 0001:00026d30       $$000000                   10027d30     MSVCRT:ftol3.obj
 0001:00026d4e       _dtol3_default             10027d4e     MSVCRT:ftol3.obj
 0001:00026d78       _dtol3_getbits             10027d78     MSVCRT:ftol3.obj
 0001:00026da1       _dtol3_trunc               10027da1     MSVCRT:ftol3.obj
 0001:00026da8       _dtol3_lshift              10027da8     MSVCRT:ftol3.obj
 0001:00026dae       _dtol3_notsafe             10027dae     MSVCRT:ftol3.obj
 0001:00026dc7       _dtol3_large               10027dc7     MSVCRT:ftol3.obj
 0001:00026dcf       _dtol3_NaN                 10027dcf     MSVCRT:ftol3.obj
 0001:00026dd7       _dtol3_retmin              10027dd7     MSVCRT:ftol3.obj
 0001:00026de0       $$000000                   10027de0     MSVCRT:ftol2.obj
 0001:00026df0       $$000000                   10027df0     MSVCRT:ftol2.obj
 0001:00026e01       L3B                        10027e01     MSVCRT:ftol2.obj
 0001:00026e44       L3F                        10027e44     MSVCRT:ftol2.obj
 0001:00026e4c       L40                        10027e4c     MSVCRT:ftol2.obj
 0001:00026e5f       L41                        10027e5f     MSVCRT:ftol2.obj
 0001:00026e6c       ?dllmain_crt_dispatch@@YGHQAUHINSTANCE__@@KQAX@Z 10027e6c f   MSVCRT:dll_dllmain.obj
 0001:00026ebf       ?dllmain_crt_process_attach@@YAHQAUHINSTANCE__@@QAX@Z 10027ebf f   MSVCRT:dll_dllmain.obj
 0001:00026fc6       ?dllmain_crt_process_detach@@YAH_N@Z 10027fc6 f   MSVCRT:dll_dllmain.obj
 0001:00027076       ?dllmain_dispatch@@YAHQAUHINSTANCE__@@KQAX@Z 10028076 f   MSVCRT:dll_dllmain.obj
 0001:00027181       ?dllmain_raw@@YGHQAUHINSTANCE__@@KQAX@Z 10028181 f   MSVCRT:dll_dllmain.obj
 0001:000273a3       ___get_entropy             100283a3 f   MSVCRT:gs_support.obj
 0001:00027492       ?find_pe_section@@YAPAU_IMAGE_SECTION_HEADER@@QAEI@Z 10028492 f   MSVCRT:utility.obj
 0001:000278f0       $$000000                   100288f0     MSVCRT:sehprolg4.obj
 0002:00000470       _TabKeys                   10029470     cmscgats.obj
 0002:00000a08       _Mantissa                  10029a08     cmshalf.obj
 0002:00002a08       _Exponent                  1002ba08     cmshalf.obj
 0002:00002b08       _Base                      1002bb08     cmshalf.obj
 0002:00002f08       _Shift                     1002bf08     cmshalf.obj
 0002:00003468       _Device2PCS16              1002c468     cmsio1.obj
 0002:00003478       _Device2PCSFloat           1002c478     cmsio1.obj
 0002:00003488       _PCS2Device16              1002c488     cmsio1.obj
 0002:00003498       _PCS2DeviceFloat           1002c498     cmsio1.obj
 0002:000034a8       _GrayInputMatrix           1002c4a8     cmsio1.obj
 0002:000034c0       _OneToThreeInputMatrix     1002c4c0     cmsio1.obj
 0002:000034d8       _PickYMatrix               1002c4d8     cmsio1.obj
 0002:000034f0       _PickLstarMatrix           1002c4f0     cmsio1.obj
 0002:00003540       ?V2ToV4@?1??_cmsStageAllocLabV2ToV4@@9@9 1002c540     cmslut.obj
 0002:00003588       ?V4ToV2@?1??_cmsStageAllocLabV4ToV2@@9@9 1002c588     cmslut.obj
 0002:000035d0       ?a1@?1??_cmsStageNormalizeFromLabFloat@@9@9 1002c5d0     cmslut.obj
 0002:00003618       ?o1@?1??_cmsStageNormalizeFromLabFloat@@9@9 1002c618     cmslut.obj
 0002:00003630       ?a1@?1??_cmsStageNormalizeFromXyzFloat@@9@9 1002c630     cmslut.obj
 0002:00003678       ?a1@?1??_cmsStageNormalizeToLabFloat@@9@9 1002c678     cmslut.obj
 0002:000036c0       ?o1@?1??_cmsStageNormalizeToLabFloat@@9@9 1002c6c0     cmslut.obj
 0002:000036d8       ?a1@?1??_cmsStageNormalizeToXyzFloat@@9@9 1002c6d8     cmslut.obj
 0002:00003828       _InputFormatters16         1002c828     cmspack.obj
 0002:00003a30       _InputFormattersFloat      1002ca30     cmspack.obj
 0002:00003a88       _OutputFormatters16        1002ca88     cmspack.obj
 0002:00003d20       _OutputFormattersFloat     1002cd20     cmspack.obj
 0002:00003eb0       _Spiral                    1002ceb0     cmssm.obj
 0002:00003f70       _SupportedTagTypes         1002cf70     cmstypes.obj
 0002:00004350       ?ParamsByType@?1??Type_ParametricCurve_Read@@9@9 1002d350     cmstypes.obj
 0002:00004364       ?ParamsByType@?1??Type_ParametricCurve_Write@@9@9 1002d364     cmstypes.obj
 0002:00004730       _AllowedLUTTypes           1002d730     cmsvirt.obj
 0002:00004950       _isotempdata               1002d950     cmswtpnt.obj
 0002:00004f70       _GS_ExceptionPointers      1002df70     MSVCRT:gs_report.obj
 0002:00004f80       _bias_low                  1002df80     MSVCRT:ftol3.obj
 0002:00004f90       _bias_high                 1002df90     MSVCRT:ftol3.obj
 0002:00004fa0       _DP2to32                   1002dfa0     MSVCRT:ftol3.obj
 0002:00004fa8       _NaN                       1002dfa8     MSVCRT:ftol3.obj
 0002:00004fac       _onept5                    1002dfac     MSVCRT:ftol3.obj
 0002:00004fb0       two32                      1002dfb0     MSVCRT:ftol2.obj
 0002:00004fb4       two63                      1002dfb4     MSVCRT:ftol2.obj
 0002:00004fb8       _NaN                       1002dfb8     MSVCRT:ftol2.obj
 0002:00005468       __sehtable$?dllmain_crt_process_attach@@YAHQAUHINSTANCE__@@QAX@Z 1002e468     MSVCRT:dll_dllmain.obj
 0002:00005488       __sehtable$?dllmain_crt_process_detach@@YAH_N@Z 1002e488     MSVCRT:dll_dllmain.obj
 0002:000054b0       __sehtable$?dllmain_dispatch@@YAHQAUHINSTANCE__@@KQAX@Z 1002e4b0     MSVCRT:dll_dllmain.obj
 0002:000054d0       __sehtable$___scrt_is_nonwritable_in_current_image 1002e4d0     MSVCRT:utility.obj
 0002:000054f0       .edata                     1002e4f0     lcms.exp
 0002:00005518       rgpv                       1002e518     lcms.exp
 0002:00005540       rgszName                   1002e540     lcms.exp
 0002:00005568       rgwOrd                     1002e568     lcms.exp
 0002:0000557c       szName                     1002e57c     lcms.exp
 0002:00005585       $N00001                    1002e585     lcms.exp
 0002:00005593       $N00002                    1002e593     lcms.exp
 0002:000055c2       $N00003                    1002e5c2     lcms.exp
 0002:000055fa       $N00004                    1002e5fa     lcms.exp
 0002:00005631       $N00005                    1002e631     lcms.exp
 0002:00005660       $N00006                    1002e660     lcms.exp
 0002:00005697       $N00007                    1002e697     lcms.exp
 0002:000056c6       $N00008                    1002e6c6     lcms.exp
 0002:000056f1       $N00009                    1002e6f1     lcms.exp
 0002:00005725       $N00010                    1002e725     lcms.exp
 0002:0000597e       .idata$6                   1002e97e     awt:awt.dll
 0002:000059c4       .idata$6                   1002e9c4     java:java.dll
 0002:00005b56       .idata$6                   1002eb56     kernel32:KERNEL32.dll
 0002:00005bbc       .idata$6                   1002ebbc     vcruntime:VCRUNTIME140.dll
 0002:00005db2       .idata$6                   1002edb2     ucrt:api-ms-win-crt-stdio-l1-1-0.dll
 0002:00005dd2       .idata$6                   1002edd2     ucrt:api-ms-win-crt-heap-l1-1-0.dll
 0002:00005df2       .idata$6                   1002edf2     ucrt:api-ms-win-crt-math-l1-1-0.dll
 0002:00005e12       .idata$6                   1002ee12     ucrt:api-ms-win-crt-string-l1-1-0.dll
 0002:00005e34       .idata$6                   1002ee34     ucrt:api-ms-win-crt-filesystem-l1-1-0.dll
 0002:00005e5a       .idata$6                   1002ee5a     ucrt:api-ms-win-crt-time-l1-1-0.dll
 0002:00005e7a       .idata$6                   1002ee7a     ucrt:api-ms-win-crt-runtime-l1-1-0.dll
 0003:00000000       ?FormattersAlpha@?1??_cmsGetFormatterAlpha@@9@9 1002f000     cmsalpha.obj
 0003:00000090       _PredefinedProperties      1002f090     cmscgats.obj
 0003:00000160       _PredefinedSampleID        1002f160     cmscgats.obj
 0003:00000208       _DefaultIntents            1002f208     cmscnvrt.obj
 0003:00000cac       ?LogErrorChunk@?1??_cmsAllocLogErrorChunk@@9@9 1002fcac     cmserr.obj
 0003:00000cb0       ?MutexChunk@?1??_cmsAllocMutexPluginChunk@@9@9 1002fcb0     cmserr.obj
 0003:00000cc0       _DefaultCurves             1002fcc0     cmsgamma.obj
 0003:00000d70       _Offset                    1002fd70     cmshalf.obj
 0003:00000df0       _DefaultOptimization       1002fdf0     cmsopt.obj
 0003:00000e10       ?RGBwhite@?1??_cmsEndPointsBySpace@@9@9 1002fe10     cmspcs.obj
 0003:00000e18       ?CMYKblack@?1??_cmsEndPointsBySpace@@9@9 1002fe18     cmspcs.obj
 0003:00000e20       ?LABblack@?1??_cmsEndPointsBySpace@@9@9 1002fe20     cmspcs.obj
 0003:00000e28       ?LABwhite@?1??_cmsEndPointsBySpace@@9@9 1002fe28     cmspcs.obj
 0003:00000e30       ?CMYblack@?1??_cmsEndPointsBySpace@@9@9 1002fe30     cmspcs.obj
 0003:00000e38       ?GrayWhite@?1??_cmsEndPointsBySpace@@9@9 1002fe38     cmspcs.obj
 0003:00000e40       _globalContext             1002fe40     cmsplugin.obj
 0003:00000e9c       __cmsContextPoolHeadMutex  1002fe9c     cmsplugin.obj
 0003:00000eb4       ?mutex@?2??cmsCreateContext@@9@9 1002feb4     cmsplugin.obj
 0003:00000eb8       _SupportedMPEtypes         1002feb8     cmstypes.obj
 0003:00000f58       _SupportedTags             1002ff58     cmstypes.obj
 0003:00002858       ?D50XYZ@?1??cmsD50_XYZ@@9@9 10031858     cmswtpnt.obj
 0003:00002898       ?AdaptationStateChunk@?1??_cmsAllocAdaptationStateChunk@@9@9 10031898     cmsxform.obj
 0003:000028a0       ?AlarmCodesChunk@?1??_cmsAllocAlarmCodesChunk@@9@9 100318a0     cmsxform.obj
 0003:000028e8       _Trans_renderType_fID      100318e8     LCMS.obj
 0003:000028ec       _Trans_ID_fID              100318ec     LCMS.obj
 0003:000028f0       _IL_isIntPacked_fID        100318f0     LCMS.obj
 0003:000028f4       _IL_dataType_fID           100318f4     LCMS.obj
 0003:000028f8       _IL_pixelType_fID          100318f8     LCMS.obj
 0003:000028fc       _IL_dataArray_fID          100318fc     LCMS.obj
 0003:00002900       _IL_offset_fID             10031900     LCMS.obj
 0003:00002904       _IL_nextRowOffset_fID      10031904     LCMS.obj
 0003:00002908       _IL_width_fID              10031908     LCMS.obj
 0003:0000290c       _IL_height_fID             1003190c     LCMS.obj
 0003:00002910       _IL_imageAtOnce_fID        10031910     LCMS.obj
 0003:00002918       ?IntentsPluginChunkType@?3??_cmsAllocIntentsPluginChunk@@9@9 10031918     cmscnvrt.obj
 0003:00002920       ?CurvesPluginChunk@?5??_cmsAllocCurvesPluginChunk@@9@9 10031920     cmsgamma.obj
 0003:00002928       ?InterpPluginChunk@?5??_cmsAllocInterpPluginChunk@@9@9 10031928     cmsintrp.obj
 0003:00002930       ?OptimizationPluginChunkType@?3??_cmsAllocOptimizationPluginChunk@@9@9 10031930     cmsopt.obj
 0003:00002938       ?FormattersPluginChunk@?5??_cmsAllocFormattersPluginChunk@@9@9 10031938     cmspack.obj
 0003:0000293c       ?RGBblack@?1??_cmsEndPointsBySpace@@9@9 1003193c     cmspcs.obj
 0003:00002944       ?CMYKwhite@?1??_cmsEndPointsBySpace@@9@9 10031944     cmspcs.obj
 0003:0000294c       ?CMYwhite@?1??_cmsEndPointsBySpace@@9@9 1003194c     cmspcs.obj
 0003:00002954       ?Grayblack@?1??_cmsEndPointsBySpace@@9@9 10031954     cmspcs.obj
 0003:0000295c       ?_cmsWindowsInitMutex@?2??cmsCreateContext@@9@9 1003195c     cmsplugin.obj
 0003:00002960       __cmsContextPoolHead       10031960     cmsplugin.obj
 0003:00002968       __cmsPSActualColumn        10031968     cmsps2.obj
 0003:00002970       ?Buffer@?1??RemoveCR@@9@9  10031970     cmsps2.obj
 0003:00003170       ?buffer@?1??EmitNGamma@@9@9 10032170     cmsps2.obj
 0003:00003970       ?buffer@?1??EmitCIEBasedDEF@@9@9 10032970     cmsps2.obj
 0003:0000417c       ?TagTypePluginChunk@?3??_cmsAllocTagTypePluginChunk@@9@9 1003317c     cmstypes.obj
 0003:00004180       ?TagTypePluginChunk@?3??_cmsAllocMPETypePluginChunk@@9@9 10033180     cmstypes.obj
 0003:00004184       ?TagPluginChunk@?3??_cmsAllocTagPluginChunk@@9@9 10033184     cmstypes.obj
 0003:00004188       ?D50xyY@?1??cmsD50_xyY@@9@9 10033188     cmswtpnt.obj
 0003:000041a4       ?TransformPluginChunkType@?3??_cmsAllocTransformPluginChunk@@9@9 100331a4     cmsxform.obj
 0003:000041a8       _GS_ExceptionRecord        100331a8     MSVCRT:gs_report.obj
 0003:000041f8       _GS_ContextRecord          100331f8     MSVCRT:gs_report.obj
 0003:000044c4       ?__proc_attached@@3HA      100334c4     MSVCRT:dll_dllmain.obj
 0003:000044e0       ?is_initialized_as_dll@@3_NA 100334e0     MSVCRT:utility.obj
 0003:000044e1       ?module_local_atexit_table_initialized@@3_NA 100334e1     MSVCRT:utility.obj
 0003:000044e4       ?module_local_atexit_table@@3U_onexit_table_t@@A 100334e4     MSVCRT:utility.obj
 0003:000044f0       ?module_local_at_quick_exit_table@@3U_onexit_table_t@@A 100334f0     MSVCRT:utility.obj
 0004:00000060       $R000000                   10034060     lcms.dll.res
